:100000000C94B7010C94A8310C94D5310C94DF01F9
:100010000C94DF010C94DF010C94DF010C94DF01E0
:100020000C94DF010C94DF010C94DF010C94CA06E0
:100030000C94DF010C94DF010C94DF010C94DF01C0
:100040000C94B4300C94DF010C9440060C947C06A4
:100050000C94DF010C94DF010C94DF010C94DF01A0
:100060000C94DF010C94DF01084AD73B3BCE016EB4
:1000700084BCBFFDC12F3D6C74319ABD56833DDAFF
:100080003D00C77F11BED9E4BB4C3E916BAAAABE0E
:10009000000000803F05A84CCDB2D44EB93836A937
:1000A000020C50B9918688083CA6AAAA2ABE000074
:1000B00000803F0664EC1B3C04BC163E3BE5B93CAB
:1000C000C93C37C29E5A3D660498083EEA69AAAA0E
:1000D0003E000000803F2020BF0020BF00BF007C0A
:1000E0002020202020202020202020202020202010
:1000F00020202000C8202020202020202020202078
:1001000020C900C8202020202020202020202020BE
:10011000C97C00D820202020202020202020202042
:10012000D97C00C820202020202020202020202032
:10013000C97C00C820202020202020202020202032
:10014000C97C00207265766F006D696E6F706F7389
:1001500064206C6962726570696C6F740020202085
:100160002020BABBBCBDBE7C2020202020CACBCC26
:10017000CDCE7C00626F6F74696E672075703AED4A
:10018000F2F2F2F2F2F2F2F30062617474657279E3
:10019000207761726E696E672000747870696420E0
:1001A00076616C756573006261726F2074656D7045
:1001B0000074656D706469737020006163746976A2
:1001C000652000706173736976650075617674618E
:1001D0006C6B200073657475702073637265656E57
:1001E0007C7C7C004368617220446F6E650A00521B
:1001F0006561647920666F7220466F6E740A0055DF
:1002000070646174652043686172536574000040D6
:100210007A10F35A00A0724E18090010A5D4E80015
:1002200000E87648170000E40B54020000CA9A3B2D
:10023000000000E1F50500008096980000004042B3
:100240000F000000A0860100000010270000000041
:10025000E803000000006400000000000A00000045
:1002600000000100000000002C76D888DC674F08F1
:1002700023DFC1DFAE59E1B1B796E5E3E453C63AF7
:10028000E651997696E8E6C28426EB898C9B62ED6E
:10029000407C6FFCEFBC9C9F40F2BAA56FA5F49028
:1002A000055A2AF75C936B6CF9676DC11BFCE0E49F
:1002B0000D47FEF520E6B500D0ED902E03009435F5
:1002C00077050080841E080000204E0A000000C848
:1002D0000C333333330F986E12831141EF8D211499
:1002E000893BE65516CFFEE6DB18D1844B381BF769
:1002F0007C1D901DA4BBE424203284725E22810008
:10030000C9F124ECA1E53D276E616E00696E6600BF
:1003100000000000240027002A0000000000250043
:1003200028002B0000000000230026002900040400
:10033000040404040404020202020202030303038D
:100340000303010204081020408001020408102069
:100350000102040810200000000700020100000351
:10036000040600000000000000004B0411081124E6
:100370001FBECFEFD8E0DEBFCDBF13E0A0E0B1E0FD
:10038000E8EFFDE602C005900D92AE3FB107D9F748
:1003900016E0AEEFB3E001C01D92A03BB107E1F75C
:1003A00013E0CEE6D3E004C02297FE010E94F636A9
:1003B000CA36D107C9F70E94BF320C94FA360C94A2
:1003C0000000FA01AA27283051F1203181F1E89488
:1003D0006F936E7F6E5F7F4F8F4F9F4FAF4FB1E038
:1003E0003ED0B4E03CD0670F781F891F9A1FA11D33
:1003F000680F791F8A1F911DA11D6A0F711D811D34
:10040000911DA11D20D009F468943F912AE0269FF8
:1004100011243019305D3193DEF6CF010895462F57
:100420004770405D4193B3E00FD0C9F7F6CF462F38
:100430004F70405D4A3318F0495D31FD40524193A1
:1004400002D0A9F7EACFB4E0A6959795879577955E
:100450006795BA95C9F700976105710508959B01E5
:10046000AC010A2E06945795479537952795BA956E
:10047000C9F7620F731F841F951FA01D08952830B0
:1004800008F027E03327DA01990F311D87FD9160CD
:1004900000966105710539F432602E5F3D9330E3BB
:1004A0002A95E1F708959F3F30F080387105610586
:1004B00009F03C5F3C5F3D93913008F08068911DEE
:1004C000DF93CF931F930F93FF92EF92192F987F93
:1004D0009695E92F96959695E90FFF27E859FD4FD8
:1004E00099273327EE24FF24A701E70105900894FC
:1004F000079428F4360FE71EF81E491F511D660F9A
:10050000771F881F991F0694A1F70590079428F478
:10051000E70EF81E491F561FC11D770F881F991F30
:10052000661F0694A1F70590079428F4F80E491F5A
:10053000561FC71FD11D880F991F661F771F06946E
:10054000A1F70590079420F4490F561FC71FD81F25
:10055000990F661F771F881F0694A9F7849110953D
:10056000177041F0D695C79557954795F794E7943E
:100570001A95C1F7EEE0F2E0689415901591359167
:100580006591959105907FE27395E118F10A430B0F
:10059000560BC90BD009C0F7E10CF11E431F561FC3
:1005A000C91FD01D7EF4703311F48A95E6CFE8940C
:1005B000015030F0080F0AF40027021708F4202F2A
:1005C0002395022F7A3328F079E37D932A95E9F772
:1005D00010C07D932A9589F606949795679537956F
:1005E00017951794E118F10A430B560BC90BD00964
:1005F00098F023957E9173957A3308F070E37C939D
:100600002013B8F77E9170617D9330F0839571E38C
:100610007D9370E32A95E1F71124EF90FF900F91FD
:100620001F91CF91DF91992787FD90950895CF93E2
:10063000DF93BC018230910510F462E070E0A0917C
:10064000AE06B091AF06ED0140E050E0E0E0F0E032
:1006500021C0888199818617970769F48A819B81D7
:10066000309719F09383828304C09093AF068093F0
:10067000AE06FE0134C06817790738F441155105FC
:1006800019F08417950708F4AC01FE018A819B815B
:100690009C01E9012097E9F641155105A9F1CA012C
:1006A000861B970B049708F4BA01E0E0F0E02AC03B
:1006B0008D919C91119784179507F9F4641775072C
:1006C00081F412968D919C911397309719F0938332
:1006D000828304C09093AF068093AE06FD013296EC
:1006E0004CC0CA01861B970BFD01E80FF91F6193EF
:1006F000719302978D939C9340C0FD0182819381F9
:100700009C01D9011097A1F68091AC069091AD069D
:10071000892B41F48091A0029091A1029093AD06A3
:100720008093AC064091A2025091A302411551055D
:1007300041F44DB75EB780919E0290919F02481B95
:10074000590B2091AC063091AD06CA01821B930B68
:100750008617970780F0AB014E5F5F4F84179507B0
:1007600050F0420F531F5093AD064093AC06F90171
:100770006193719302C0E0E0F0E0CF01DF91CF918F
:100780000895CF93DF93009709F450C0EC012297AE
:100790001B821A82A091AE06B091AF06109709F1A4
:1007A00040E050E0AC17BD0708F1BB83AA83FE010F
:1007B00021913191E20FF31FAE17BF0779F48D91AC
:1007C0009C911197280F391F2E5F3F4F3983288343
:1007D00012968D919C9113979B838A8341155105A5
:1007E00071F4D093AF06C093AE0620C012968D91DF
:1007F0009C911397AD01009711F0DC01D3CFFA0162
:10080000D383C28321913191E20FF31FCE17DF070B
:1008100069F488819981280F391F2E5F3F4FFA01B3
:10082000318320838A819B8193838283DF91CF915F
:100830000895FC010590615070400110D8F7809533
:1008400090958E0F9F1F0895FC016150704001909C
:100850000110D8F7809590958E0F9F1F08956EBD5B
:100860000DB407FEFDCF8EB508958DE061E00E94C6
:1008700002328BE061E00E9402328CE060E00E9474
:1008800002328AE061E00E9402321CBC80E58CBD2D
:100890008DB58EB508958EEF93E00E9435040895CE
:1008A000FC011382128288EE93E0A0E0B0E0848322
:1008B0009583A683B78384EB92E091838083089528
:1008C000FC018089803419F421E030E002C020E08E
:1008D00030E0C9010895FC01818990E00895FC0190
:1008E0006487458766874787089580E090E008958C
:1008F00080E090E0089580E090E008950895EF9200
:10090000FF921F93CF93DF93162F7A0186E060E06A
:100910000E9441328EEF93E060E00E942F048EEF40
:1009200093E060E00E942F048EEF93E069E00E9464
:100930002F048EEF93E0612F0E942F04C0E0D0E0DF
:10094000F701EC0FFD1F10818EEF93E06AE00E942B
:100950002F048EEF93E06C2F0E942F048EEF93E014
:100960006BE00E942F048EEF93E0612F0E942F0412
:100970002196C633D10521F78EEF93E068E00E94FF
:100980002F048EEF93E060EA0E942F048EEF93E035
:1009900060EA0E942F0485FDF9CF8EEF93E060E0BE
:1009A0000E942F048EEF93E06CE00E942F0486E0FB
:1009B00061E00E944132DF91CF911F91FF90EF9053
:1009C00008951F93CF93DF93EC01162F86E060E02C
:1009D0000E9441328EEF93E060E00E942F041123C9
:1009E00019F0113059F404C08EEF93E0688904C007
:1009F00068896C618EEF93E00E942F0486E061E0CD
:100A00000E944132DF91CF911F910895EF92FF92A2
:100A10000F931F938EE1489F70011124E60EF11C85
:100A200086E060E00E9441320EEF13E0C80165E00D
:100A30000E942F04C8016F2D0E942F04C80166E098
:100A40000E942F04C8016E2D0E942F041F910F9148
:100A5000FF90EF900895EF92FF920F931F937C0108
:100A60000EEF13E0C80167E00E942F04C8016FEF8A
:100A70000E942F0486E061E00E944132F7018785E1
:100A80008F5F87871F910F91FF90EF900895EF92EE
:100A9000FF920F931F93FC01E7848EE1E89E7001A3
:100AA00011248685E80EF11C86E060E00E94413248
:100AB0000EEF13E0C80164E00E942F04C80163E058
:100AC0000E942F04C80165E00E942F04C8016F2D09
:100AD0000E942F04C80166E00E942F04C8016E2DF9
:100AE0000E942F041F910F91FF90EF9008951F9384
:100AF000CF93DF93EC01162F6C3731F40E942B0556
:100B0000CE010E9447050AC08EEF93E067E00E9485
:100B10002F048EEF93E0612F0E942F0481E090E07C
:100B2000DF91CF911F9108950F931F9386E060E0AE
:100B30000E9441320EEF13E0C80164E00E942F04CE
:100B4000C80164E00E942F0486E061E00E94413207
:100B50001F910F9108951F93CF93DF93EC01188A93
:100B600016E0198B8CE996E060E973E00E9414307E
:100B7000813049F480E4888B88E0898B86E060E0EE
:100B80000E94413202C0188A198B86E060E00E9400
:100B90004132DF91CF911F9108950F931F93CF930F
:100BA000DF93EC0186E061E00E94023282E060E0C7
:100BB0000E94023282E061E00E944132CE010E9436
:100BC000AB0586E060E00E9441328EEF93E06CEE70
:100BD0000E942F048EEF93E06FEF0E942F04182FD6
:100BE0008EEF93E060E00E942F04688962608EEFD0
:100BF00093E00E942F0462E370E080E090E00E94A6
:100C00000A318EEF93E06CE60E942F041F7E8EEF78
:100C100093E0612F0E942F048889803419F00DE041
:100C200010E002C000E110E0109200041092FF03F7
:100C300017C06091FF0370910004605F8EEF93E036
:100C40000E942F048EEF93E069E00E942F048091B0
:100C5000FF03909100040196909300048093FF039A
:100C60008091FF03909100048017910714F3CE0147
:100C700061E00E94E104DF91CF911F910F910895EF
:100C80001F920F920FB60F9211242F933F934F9301
:100C90008F939F93EF93FF934091C60020918B0613
:100CA00030918C062F5F3F4F80918F069091900678
:100CB0002823392380918D0690918E0628173907B5
:100CC00079F080918B0690918C06E0919106F091DD
:100CD0009206E80FF91F408330938C0620938B0611
:100CE000FF91EF919F918F914F913F912F910F9095
:100CF0000FBE0F901F9018951F920F920FB60F9274
:100D000011242F933F938F939F93EF93FF93209101
:100D10009506309196068091930690919406281737
:100D20003907E9F08091950690919606E091990631
:100D3000F0919A06E80FF91F80818093C600809198
:100D40009506909196060196209197063091980607
:100D500082239323909396068093950610C020914A
:100D600093063091940680919506909196062817E7
:100D7000390729F48091C1008F7D8093C100FF91D4
:100D8000EF919F918F913F912F910F900FBE0F90F8
:100D90001F9018951F920F920FB60F9211248F93E8
:100DA0009F938091C1049091C204892B51F080914E
:100DB000C3049091C40401969093C4048093C30427
:100DC00009C08091C5049091C60401969093C60411
:100DD0008093C5049F918F910F900FBE0F901F902D
:100DE0001895CF93DF93482FEB0180912206833033
:100DF00009F45DC0843028F48130C1F0823058F5A8
:100E00000AC0853009F4D2C0853008F4A8C0863005
:100E100009F0F2C0E9C04C3309F0EEC081E08093E4
:100E20002206488384EB80932106E6C0842F90E05D
:100E3000E0912106F0E0E827F927EE53FD4F2081ED
:100E400020932106887F9070809741F582E08093FF
:100E50002206498329C0242F30E0E0912106F0E0EA
:100E6000E227F327EE53FD4F808180932106809186
:100E700020068F5F80932006823018F43B832A83FC
:100E8000BBC0922F88272A813B81820F931F9B83AF
:100E90008A830A978F3F910521F018F0109222065D
:100EA000ABC083E08093220610922006A5C0E42FF9
:100EB000F0E08091210690E0E827F927EE53FD4FFE
:100EC000808180932106609120066F5F60932006E9
:100ED000623089F0633020F4613009F08DC006C0C3
:100EE000633091F0643009F087C022C0842F90E015
:100EF000A0E0B0E018C0242F30E040E050E0542FD4
:100F0000432F322F222707C0242F30E040E050E04B
:100F1000A901332722278C819D81AE81BF81820F59
:100F2000931FA41FB51F8C839D83AE83BF8364C0B2
:100F3000242F30E040E050E0522F4427332722276F
:100F40008C819D81AE81BF81820F931FA41FB51F2D
:100F50008C839D83AE83BF8360932206A5CF242F0D
:100F600030E0E0912106F0E0E227F327EE53FD4F59
:100F7000808180932106809120068F5F80932006D8
:100F8000813019F08230C1F503C03987288734C019
:100F9000922F882728853985280F391F3987288778
:100FA0008A819B810A97F1F085E07CCFE42FF0E005
:100FB0008091210690E0E827F927EE53FD4F8081CC
:100FC00080932106209120062F5F2093200630E099
:100FD000FB01E20FF31F41878A819B810A97281743
:100FE000390750F086E05ECFC75FDE4F4883C950B7
:100FF000D14087E08093220680912206873069F4F1
:1010000010922206C75FDE4F909121068881C95059
:10101000D140981711F48A8101C080E0DF91CF910F
:1010200008958F92AF92CF92EF92FF920F931F93FA
:1010300087E894E060E045EC50E024EC30E000EC20
:1010400010E0B1ECEB2EF12CCC24C394A8E9AA2E2D
:10105000F0E28F2E0E94842984EA94E00E945004DA
:101060001092B7041092B8041092B9041092BA0406
:101070001092BB041092BC041092BD041092BE04E6
:101080001092C0041092BF041092B6041F910F91E9
:10109000FF90EF90CF90AF908F900895AF92BF9256
:1010A000CF92DF92EF92FF920F931F93E09087060B
:1010B000F09088060091890610918A068FE590E0ED
:1010C000A0E0B0E0E80EF91E0A1F1B1F0E94FC30D2
:1010D0006E157F058007910708F44EC0A090EC04C0
:1010E000B090ED04C090EE04D090EF04C601B501BD
:1010F00020E030E040E85FE30E945F35181694F589
:10110000E0903F06F09040060091410610914206A3
:101110000E94FC3020918706309188064091890614
:1011200050918A06621B730B840B950B0E94353419
:101130009B01AC01C601B5010E946A3520E030E098
:101140004AE754E40E949C339B01AC01C801B701FB
:101150000E94CF3260933F06709340068093410611
:10116000909342060E94FC30609387067093880635
:101170008093890690938A061F910F91FF90EF90BC
:10118000DF90CF90BF90AF900895DF93CF9300D0C2
:1011900000D0CDB7DEB7FB01E80FF91F628583856C
:1011A0009485258569838A839B832C83492F5C8161
:1011B000782FCA010F900F900F900F90CF91DF9171
:1011C0000895AF92BF92DF92EF92FF920F931F9319
:1011D000CF93DF938C018091230680FDE4C0F8015A
:1011E000F08087E894E06F2D0E94652AE801C75FD0
:1011F000DE4FEF2DF0E0EE53FD4F80818883F80144
:10120000F18087E894E06F2D0E94652AEF2DF0E0D1
:10121000888190E0E827F927EE53FD4F808188838D
:10122000F801F28087E894E06F2D0E94652AEF2D87
:10123000F0E0888190E0E827F927EE53FD4F8081A8
:101240008883F801F38087E894E06F2D0E94652A77
:10125000EF2DF0E0888190E0E827F927EE53FD4F6D
:1012600080818883F801F48087E894E06F2D0E94E4
:10127000652AEF2DF0E0888190E0E827F927EE530A
:10128000FD4F80818883F801248135814681578113
:10129000232F342F452F5527F22E87E894E0622F15
:1012A0000E94652AEF2DF0E0888190E0E827F92779
:1012B000EE53FD4F80818883F8012481358146817A
:1012C00057819A0144275527F22E87E894E0622F30
:1012D0000E94652AEF2DF0E0888190E0E827F92749
:1012E000EE53FD4F80818883F8012481358146814A
:1012F0005781252F332744275527F22E87E894E07E
:10130000622F0E94652AEF2DF0E0888190E0E827A7
:10131000F927EE53FD4F8081888387E894E060E0F1
:101320000E94652AE881F0E0EE53FD4F80818883BA
:1013300087E894E060E00E94652AE881F0E0EE53DF
:10134000FD4F80818883F801828193810B9718F18A
:101350008AE0A82EB12CA00EB11E750112C0F701B3
:10136000D1907F0187E894E06D2D0E94652AED2DD4
:10137000F0E0888190E0E827F927EE53FD4F808167
:1013800088832E2D2A1930E0F801828193810A97F3
:101390002817390720F3075F1E4F87E894E0F8010C
:1013A00060810E94652ADF91CF911F910F91FF907C
:1013B000EF90DF90BF90AF900895DF93CF93CDB7BC
:1013C000DEB7CA50D1400FB6F894DEBF0FBECDBF16
:1013D0002CE329836A832AE030E03C832B83FC01E1
:1013E00084819581A681B7818D839E83AF83B887E1
:1013F000CE0101960E94E108C65FDE4F0FB6F89459
:10140000DEBF0FBECDBFCF91DF9108958CE996E08E
:101410006AE773E00E941430882331F586E696E689
:10142000A6E6B0E48093240690932506A0932606B2
:10143000B093270680E090E0A0E8BFE38093280601
:1014400090932906A0932A06B0932B0688EE93E08A
:1014500090932D0680932C0681E880932E068DE8CC
:1014600080932F068DEF25C082E598EBAEE0B0E4C7
:101470008093240690932506A0932606B093270612
:1014800085E89BEEA1E5B0E48093280690932906B9
:10149000A0932A06B0932B0680EA94E190932D0640
:1014A00080932C068BEF80932E0686E680932F0682
:1014B0008AEF809330060895FF920F931F930CE9F3
:1014C00016E0C8016CE773E00E94143080936B064D
:1014D000C8016EE773E00E94143080936C06C80167
:1014E00060E873E00E94143080934B06C8016EE8F8
:1014F00073E00E94143080936306C8016AE873E0C9
:101500000E94143080936106C80164E873E00E9471
:10151000143080936D06C80166E873E00E941430B1
:1015200080936E06C8016CE873E00E9414308093CB
:101530005306C80162E973E00E94143080936F067D
:10154000C80164E973E00E94143080935206C80118
:1015500064EF73E00E941430F82EC80165EF73E069
:101560000E941430382F20E02F0D311D309371066A
:1015700020937006C80166EF73E00E941430F82EC5
:10158000C80167EF73E00E941430382F20E02F0D60
:10159000311D3093730620937206C80168EF73E023
:1015A0000E941430F82EC80169EF73E00E941430D5
:1015B000382F20E02F0D311D3093750620937406CF
:1015C000C8016BEF73E00E94143080934A061F91AC
:1015D0000F91FF900895BC018CE996E00E941430B1
:1015E00008956091D6047091D7048091D8049091A9
:1015F000D90420E030E040E152E40E946A3520E066
:1016000030E044EB53E40E949C330E94CD350E94AD
:1016100004349B012550304037FF03C09B01215EFD
:101620003F4FA3E3B6E0F901EE53FC4F80818C936A
:101630002F5F3F4F2432310514F020E030E0119647
:1016400086E0AE33B80779F71C9208952F923F9247
:101650004F925F926F927F928F929F92AF92BF92C2
:10166000CF92DF92EF92FF920F931F93DF93CF936E
:1016700000D000D000D0CDB7DEB7182F662E209155
:10168000CC043091CD042A35310530F0C9018D5498
:101690009F4F89359105E8F437FF02C02D543F4F25
:1016A000C90137FF03C0909581959F4F8A319105FD
:1016B0003CF0F4E48F2E912CE9ED2E2E312C1DC040
:1016C0000A975CF17BE3872E912C62ED262E312C5C
:1016D00020C02B35310514F0235B3040C90137FFA2
:1016E00003C0909581959F4F8A31910554F056E53E
:1016F000852E912C4CED242E312C37E0A32EB12CCD
:1017000015C00A9754F02DE4822E912C94ED292EC9
:10171000312C88E0A82EB12C09C005E0802E912C38
:10172000B8E32B2E312CA9E0AA2EB12C6091CE0467
:101730007091CF04882777FD8095982F0E943734C9
:1017400027EA32E94BE25CEB0E946A350E943E36A2
:1017500020E030E040EA50E40E946A3520E030E0CA
:1017600040E951E40E946A350E94CD3520E030E026
:1017700044E352E40E94CF320E940434712EFEEB07
:10178000CF2EFFEFDF2E9B01442737FD4095542FCE
:1017900029833A834B835C83E4EA4E2EE4E05E2E99
:1017A0004AEF5FEF240E351E6091CC047091CD049A
:1017B000882777FD8095982F0E94373425E33AEFEC
:1017C0004EE85CE30E946A350E943E367B018C0144
:1017D000B601882777FD8095982F0E9437349B01AA
:1017E000AC01C801B7010E946A357B018C01698197
:1017F0007A818B819C810E9437349B01AC01C801A6
:10180000B7010E94CF320E9404349B01CB010197A3
:101810008A35910508F071C062E170E00E94A4363B
:101820008B012F5F3F4FAEEEBFEF6A9FC0016B9FF2
:10183000900D7A9F900D1124820F931F62E070E04B
:101840000E94A4366D837E83E62CE01A4E2D4C5FF9
:1018500084EA94E0672D0E94060500D000D000D0F5
:10186000EDB7FEB73196ADB7BEB712965C924E9209
:10187000119720E031E0338322838D819E81880D92
:10188000991D958384830E9463294DB75EB74A5F93
:101890005F4F0FB6F8945EBF0FBE4DBF8D819E8126
:1018A0008A159B0554F1043011053CF593E0E90ECF
:1018B000C201672D4E2D0E94060500D000D000D039
:1018C000EDB7FEB73196ADB7BEB712965C924E92A9
:1018D000119720E031E0338322834D815E81420DF8
:1018E000531D558344830E9463298DB79EB7069686
:1018F0000FB6F8949EBF0FBE8DBFACE0B0E0CA0E2D
:10190000DB1E7394BEE4CB16D10409F04DCF2696AE
:101910000FB6F894DEBF0FBECDBFCF91DF911F9100
:101920000F91FF90EF90DF90CF90BF90AF909F907E
:101930008F907F906F905F904F903F902F90089581
:10194000823010F422E002C0282F220F30E08DB741
:101950009EB708970FB6F8949EBF0FBE8DBFEDB728
:10196000FEB7319684EA94E0ADB7BEB712969C9369
:101970008E93119783E091E09383828322573F4FA8
:10198000358324832F5F3F4F378326830E9463294B
:101990008DB79EB708960FB6F8949EBF0FBE8DBF49
:1019A0000895CF93DF93AC01E091DE04F091DF0462
:1019B0002091310630913206C9018C599F4F8E1704
:1019C0009F071CF4EA01219709C024563040E21712
:1019D000F30714F0EA0102C0EA012196842F90E097
:1019E000C817D90729F08CE996E04C2F0E941B30CC
:1019F000CE01DF91CF9108950F931F930CE916E06C
:101A0000C80163EF73E041E00E941B30C80164EF3E
:101A100073E043E10E941B30C80165EF73E046E0CC
:101A20000E941B30C80166EF73E040E10E941B304A
:101A3000C80167EF73E047E20E941B30C80168EFFE
:101A400073E048E80E941B30C80169EF73E043E18E
:101A50000E941B301F910F910895CF92DF92EF9259
:101A6000FF920F931F937C01D62EC72E04EA14E039
:101A7000C8016E2D4D2D0E946F04C8010E944705BC
:101A800000D000D0EDB7FEB71283018383E391E06D
:101A9000948383830E945229EDB7FEB7128301839A
:101AA00083E291E0948383830E945229EDB7FEB7CD
:101AB0001283018383E191E0948383830E945229FE
:101AC000EDB7FEB71283018383E091E094838383B3
:101AD0000E945229EDB7FEB71283018384EF90E094
:101AE000948383830E9452290F900F900F900F9040
:101AF000C8010E942B05C70101966D2D7C2D0E9407
:101B0000260B1F910F91FF90EF90DF90CF900895DB
:101B1000AF92BF92CF92DF92EF92FF920F931F93FB
:101B2000B82EA62E0E94FC3028EE33E040E050E0B4
:101B30000E94B73679018A01A4EACA2EA4E0DA2EFF
:101B4000C6016B2D4A2D0E946F04C6010E944705F5
:101B5000A090FC04B090FD048DB79EB744970FB6DB
:101B6000F8949EBF0FBE8DBFEDB7FEB73196ADB7EF
:101B7000BEB71296DC92CE92119788E091E09383E3
:101B8000828383EB90E095838483C7016CE370E0EC
:101B90000E94A436CB016CE370E00E94A4369783C8
:101BA00086832AE330E031872087C7016CE370E049
:101BB0000E94A4369387828785E690E09587848784
:101BC000C5016CE370E00E949036CB016CE370E0DD
:101BD0000E94A43697878687318B208BC5016CE3E2
:101BE00070E00E949036938B828B0E9463298DB7A0
:101BF0009EB744960FB6F8949EBF0FBE8DBFC60128
:101C00000E942B051F910F91FF90EF90DF90CF90D6
:101C1000BF90AF900895EF92FF920F931F93282FDC
:101C2000462FB4EAEB2EB4E0FB2EC701622F0E94D0
:101C30006F04C7010E9447058DB79EB70A970FB67C
:101C4000F8949EBF0FBE8DBF0DB71EB70F5F1F4F1D
:101C5000EDB7FEB7F282E18280E291E0F801938372
:101C600082836091FE047091FF0480910005909141
:101C70000105209128063091290640912A065091AD
:101C80002B060E946A35F8016483758386839783E7
:101C900080EB90E0918780870E9463298DB79EB783
:101CA0000A960FB6F8949EBF0FBE8DBFC7010E9463
:101CB0002B051F910F91FF90EF9008958F929F92A7
:101CC000AF92BF92CF92DF92EF92FF920F931F934A
:101CD000E82EF62E04EA14E0C8016E2D4F2D0E9466
:101CE0006F04C8010E9447058DB79EB70C970FB6C9
:101CF000F8949EBF0FBE8DBFEDB7FEB73196ADB75E
:101D0000BEB712961C930E93119728E2822E21E003
:101D1000922E938282829DEEA92EB12CB582A4824E
:101D20008091070590910805A0910905B0910A05D9
:101D300086839783A087B18783EFC82ED12CD38663
:101D4000C2860E9463298DB79EB70C960FB6F89491
:101D50009EBF0FBE8DBFC8010E942B05F394C80122
:101D60006E2D4F2D0E946F04C8010E944705ADB72C
:101D7000BEB71C970FB6F894BEBF0FBEADBFEDB790
:101D8000FEB7319612961C930E931197938282821E
:101D9000B582A48280910B0590910C05A0910D0550
:101DA000B0910E0586839783A087B187D386C286BC
:101DB0000E9463298DB79EB70C960FB6F8949EBF0C
:101DC0000FBE8DBFC8010E942B05F394C8016E2D74
:101DD0004F2D0E946F04C8010E944705ADB7BEB7E2
:101DE0001C970FB6F894BEBF0FBEADBFEDB7FEB7E0
:101DF000319612961C930E93119793828282B5822C
:101E0000A48280910F0590911005A0911105B091C9
:101E1000120586839783A087B187D386C2860E94E6
:101E200063298DB79EB70C960FB6F8949EBF0FBE70
:101E30008DBFC8010E942B051F910F91FF90EF905D
:101E4000DF90CF90BF90AF909F908F9008950F93A9
:101E50001F93282F462F04EA14E0C801622F0E9426
:101E60006F04C8010E9447058DB79EB70A970FB649
:101E7000F8949EBF0FBE8DBFEDB7FEB73196ADB7DC
:101E8000BEB712961C930E93119782E391E0938351
:101E9000828389EB90E0958384838091FA0490910A
:101EA000FB049783868382E890E0918780870E9475
:101EB00063298DB79EB70A960FB6F8949EBF0FBEE2
:101EC0008DBFC8010E942B051F910F910895EF92BD
:101ED000FF920F931F93282F462F34EAE32E34E00E
:101EE000F32EC701622F0E946F04C7010E944705AD
:101EF0008DB79EB70C970FB6F8949EBF0FBE8DBFDF
:101F00000DB71EB70F5F1F4FEDB7FEB7F282E1822C
:101F10008AE391E0F8019383828384EE90E09583D5
:101F200084836091F8047091F904882777FD809587
:101F3000982F0E9437342AE037ED43E25CE30E9499
:101F40006A35F80166837783808791878FE890E010
:101F5000938782870E9463298DB79EB70C960FB630
:101F6000F8949EBF0FBE8DBFC7010E942B051F9125
:101F70000F91FF90EF9008950F931F93282F462FF6
:101F800004EA14E0C801622F0E946F04C8010E9495
:101F900047058DB79EB70C970FB6F8949EBF0FBE3E
:101FA0008DBFEDB7FEB73196ADB7BEB712961C9395
:101FB0000E9311978AE391E09383828382EE90E0FF
:101FC000958384838091F4049091F504A091F604A4
:101FD000B091F70486839783A087B1878EE890E05D
:101FE000938782870E9463298DB79EB70C960FB6A0
:101FF000F8949EBF0FBE8DBFC8010E942B051F9194
:102000000F9108950F931F93282F462F84EA94E091
:10201000622F0E946F0484EA94E00E944705809139
:10202000DB04882319F424E431E057C0813019F42B
:1020300028E431E052C0823019F42CE431E04DC084
:10204000833019F420E531E048C0843019F424E5E8
:1020500031E043C0853019F428E531E03EC08630D8
:1020600019F42CE531E039C0873019F420E631E06D
:1020700034C0883019F424E631E02FC0893019F4D7
:1020800028E631E02AC08A3019F42CE631E025C078
:102090008B3019F420E731E020C08C3019F424E7AC
:1020A00031E01BC08D3019F428E731E016C08E30C6
:1020B00019F42CE731E011C08F3019F420E831E039
:1020C0000CC0803119F424E831E007C0813119F0E7
:1020D00028E831E002C029E831E08DB79EB70897C3
:1020E0000FB6F8949EBF0FBE8DBFEDB7FEB7319609
:1020F00004EA14E0ADB7BEB712961C930E93119785
:102100008DE891E09383828380EE90E095838483D1
:10211000378326830E9463298DB79EB708960FB632
:10212000F8949EBF0FBE8DBFC8010E942B051F9162
:102130000F9108950F931F93282F462F04EA14E060
:10214000C801622F0E946F04C8010E9447058DB725
:102150009EB70A970FB6F8949EBF0FBE8DBFEDB71E
:10216000FEB73196ADB7BEB712961C930E9311977A
:1021700082E991E09383828387E890E0958384836A
:102180008091DC049091DD049783868385E290E062
:10219000918780870E9463298DB79EB70A960FB6F4
:1021A000F8949EBF0FBE8DBFC8010E942B051F91E2
:1021B0000F9108950F931F93282F462F04EA14E0E0
:1021C000C801622F0E946F04C8010E9447058DB7A5
:1021D0009EB70A970FB6F8949EBF0FBE8DBFEDB79E
:1021E000FEB73196ADB7BEB712961C930E931197FA
:1021F0008CE991E0938382838091CE049091CF0407
:102200009583848380EB90E09783868381EB90E0D5
:10221000918780870E9463298DB79EB70A960FB673
:10222000F8949EBF0FBE8DBFC8010E942B051F9161
:102230000F9108950F931F93282F462F04EA14E05F
:10224000C801622F0E946F04C8010E9447058DB724
:102250009EB70A970FB6F8949EBF0FBE8DBFEDB71D
:10226000FEB73196ADB7BEB712961C930E93119779
:102270008CE991E0938382838091CC049091CD048A
:102280009583848380EB90E09783868382EB90E054
:10229000918780870E9463298DB79EB70A960FB6F3
:1022A000F8949EBF0FBE8DBFC8010E942B051F91E1
:1022B0000F9108950F931F93282F462F04EA14E0DF
:1022C000C801622F0E946F04C8010E9447058DB7A4
:1022D0009EB70A970FB6F8949EBF0FBE8DBFEDB79D
:1022E000FEB73196ADB7BEB712961C930E931197F9
:1022F00084EA91E09383828381EE90E095838483E6
:102300008091AC029091AD029783868385E290E044
:10231000918780870E9463298DB79EB70A960FB672
:10232000F8949EBF0FBE8DBFC8010E942B051F9160
:102330000F9108950F931F93282F462F04EA14E05E
:10234000C801622F0E946F04C8010E9447058DB723
:102350009EB70C970FB6F8949EBF0FBE8DBFEDB71A
:10236000FEB73196ADB7BEB712961C930E93119778
:102370008CEA91E09383828386EB91E0958384835A
:1023800080ED90E09783868383E396E09187808752
:1023900081ED90E0938782870E9463298DB79EB775
:1023A0000C960FB6F8949EBF0FBE8DBFC8010E9459
:1023B0002B051F910F9108950F931F93282F462FE0
:1023C00004EA14E0C801622F0E946F04C8010E9451
:1023D00047058DB79EB70A970FB6F8949EBF0FBEFC
:1023E0008DBFEDB7FEB73196ADB7BEB712961C9351
:1023F0000E93119784EC91E0938382838091D604AD
:102400009091D704A091D804B091D9048483958386
:10241000A683B78380EB90E0918780870E94632931
:102420008DB79EB70A960FB6F8949EBF0FBE8DBFAC
:10243000C8010E942B051F910F9108950F931F93C0
:10244000282F462F04EA14E0C801622F0E946F046F
:10245000C8010E9447058DB79EB70C970FB6F89438
:102460009EBF0FBE8DBFEDB7FEB73196ADB7BEB7FD
:1024700012961C930E9311978CEC91E093838283B8
:1024800086E190E0958384838091F0049091F1043B
:10249000A091F204B091F30486839783A087B1875B
:1024A00088E890E0938782870E9463298DB79EB762
:1024B0000C960FB6F8949EBF0FBE8DBFC8010E9448
:1024C0002B051F910F910895CF92DF92EF92FF920B
:1024D0000F931F93CF93DF93282F462FC4EAD4E0A6
:1024E000CE01622F0E946F04CE010E9447056091C9
:1024F0003F067091400680914106909142062091DE
:1025000028063091290640912A0650912B060E94F8
:102510006A356B017C0120E030E04AE754E40E9418
:102520005F351816D4F58DB79EB70C970FB6F89493
:102530009EBF0FBE8DBF0DB71EB70F5F1F4FADB74C
:10254000BEB71296DC93CE9311978AE391E0F8011F
:10255000938382838EEF90E09583848360912C0631
:1025600070912D06882777FD8095982F0E9437342B
:102570009B01AC01C701B6010E949C33D80116969D
:102580006D937D938D939C931997809130061A9645
:102590008C931A971B961C9221C08DB79EB70C97EF
:1025A0000FB6F8949EBF0FBE8DBFEDB7FEB7319644
:1025B000ADB7BEB71296DC93CE93119786ED91E03E
:1025C000938382838EEF90E095838483C682D78243
:1025D000E086F18680912F06828713860E94632908
:1025E000EDB7FEB73C960FB6F894FEBF0FBEEDBF39
:1025F00084EA94E00E942B05DF91CF911F910F9107
:10260000FF90EF90DF90CF900895EF92FF920F939D
:102610001F93282F462F54EAE52E54E0F52EC701CC
:10262000622F0E946F04C7010E9447058DB79EB7B5
:102630000C970FB6F8949EBF0FBE8DBF0DB71EB797
:102640000F5F1F4FEDB7FEB7F282E1828CEC91E095
:10265000F8019383828389EE90E09583848360916F
:10266000EC047091ED048091EE049091EF042091C0
:1026700024063091250640912606509127060E9497
:102680006A35F801668377838087918780912E066B
:10269000828713860E9463298DB79EB70C960FB66A
:1026A000F8949EBF0FBE8DBFC7010E942B051F91DE
:1026B0000F91FF90EF900895EF92FF920F931F9369
:1026C000282F462F64EAE62E64E0F62EC701622F1B
:1026D0000E946F04C7010E9447058DB79EB70C97F3
:1026E0000FB6F8949EBF0FBE8DBF0DB71EB70F5F1C
:1026F0001F4FEDB7FEB7F282E18286ED91E0F8015F
:102700009383828386EE90E0958384836091E804CE
:102710007091E9048091EA049091EB0420912806DD
:102720003091290640912A0650912B060E946A3565
:10273000F801668377838087918780912F0682874F
:1027400013860E9463298DB79EB70C960FB6F89436
:102750009EBF0FBE8DBFC7010E942B051F910F9119
:10276000FF90EF900895EF92FF920F931F93282F01
:10277000462F74EAE72E74E0F72EC701622F0E94FD
:102780006F04C7010E9447058DB79EB70C970FB61F
:10279000F8949EBF0FBE8DBF0DB71EB70F5F1F4FC2
:1027A000EDB7FEB7F282E18286ED91E0F801938306
:1027B000828387EE90E09583848360910205709117
:1027C0000305882777FD8095982F0E943734209144
:1027D00028063091290640912A0650912B060E9426
:1027E0006A35F801668377838087918780912F0609
:1027F000828713860E9463298DB79EB70C960FB609
:10280000F8949EBF0FBE8DBFC7010E942B051F917C
:102810000F91FF90EF9008950F931F93282F462F4D
:1028200004EA14E0C801622F0E946F04C8010E94EC
:102830004705809143060E94A00CC8010E942B0509
:102840001F910F910895EF92FF920F931F93282FDE
:10285000462FE4EAEE2EE4E0FE2EC701622F0E942E
:102860006F04C7010E9447058DB79EB70C970FB63E
:10287000F8949EBF0FBE8DBF0DB71EB70F5F1F4FE1
:10288000EDB7FEB7F282E18286ED91E0F801938325
:1028900082838FE190E095838483609144067091F8
:1028A000450680914606909147060E943734209154
:1028B00028063091290640912A0650912B060E9445
:1028C0006A35F801668377838087918780912F0628
:1028D000828713860E9463298DB79EB70C960FB628
:1028E000F8949EBF0FBE8DBFC7010E942B051F919C
:1028F0000F91FF90EF9008950F931F93282F462F6D
:1029000004EA14E0C801622F0E946F04C8010E940B
:1029100047058DB79EB740970FB6F8949EBF0FBE80
:102920008DBFEDB7FEB73196ADB7BEB712961C930B
:102930000E93119780EE91E09383828383E890E079
:10294000958384838091D2049091D304A091D40480
:10295000B091D50486839783A087B18784E890E0FF
:10296000938782878091E2049091E304A091E4042C
:10297000B091E50484879587A687B7870E9463296D
:102980008DB79EB740960FB6F8949EBF0FBE8DBF11
:10299000C8010E942B051F910F9108950F931F935B
:1029A000282F462F84EA94E0622F0E946F0484EA65
:1029B00094E00E9447058091E704282F30E08230A0
:1029C00030F4F4E0220F331FFA95E1F702C02150F2
:1029D000304000D000D000D0EDB7FEB7319604EA09
:1029E00014E0ADB7BEB712961C930E93119780E01A
:1029F00091E093838283358324830E9463298DB77A
:102A00009EB706960FB6F8949EBF0FBE8DBFC80145
:102A10000E942B051F910F9108950F931F93282F4C
:102A2000462F04EA14E0C801622F0E946F04C80117
:102A30000E9447058DB79EB708970FB6F8949EBFC2
:102A40000FBE8DBFEDB7FEB73196ADB7BEB71296CC
:102A50001C930E93119782EF91E0938382838FE012
:102A600090E0958384838091E604868317820E9498
:102A700063298DB79EB708960FB6F8949EBF0FBE18
:102A80008DBFC8010E942B051F910F9108950F93D0
:102A90001F9304EA14E0C80163E045E00E946F045C
:102AA000C8010E94470500D000D0EDB7FEB71283E1
:102AB00001838DE591E0948383830E945229EDB7D1
:102AC000FEB71283018389E491E0948383830E949B
:102AD0005229EDB7FEB71283018383E491E094831A
:102AE00083830E9452290F900F900F900F90C8017E
:102AF0000E942B051F910F9108950F931F93282F6C
:102B0000462F04EA14E0C801622F0E946F04C80136
:102B10000E94470500D000D0EDB7FEB712830183B5
:102B200084E791E0948383830E9452290F900F9051
:102B30000F900F90C8010E942B051F910F910895CF
:102B4000EF92FF920F931F93CF93DF930E94FC307D
:102B500020914D0630914E0640914F0650915006FF
:102B6000261737074807590708F08AC10E94FC302A
:102B70006C507E4F8F4F9F4F60934D0670934E0663
:102B800080934F069093500604EA14E0C8010E9417
:102B90009405C80165E043E00E946F04C8010E94EB
:102BA000470500D000D0EDB7FEB71283018384ED56
:102BB00091E0948383830E9452290F900F900F908D
:102BC0000F908091310690913206892B31F08091DF
:102BD000480690914906892B81F48091DE049091FA
:102BE000DF0490933206809331068091E004909147
:102BF000E10490934906809348062091E0043091C7
:102C0000E1044091480650914906C901845690401C
:102C10004817590724F480914C068F5F08C02C593F
:102C20003F4F241735072CF480914C068150809338
:102C30004C0680914C06181614F081E003C08430D5
:102C40001CF083E080934C0680914C06823009F49E
:102C500062C0833009F4BEC0813009F00DC100D0DC
:102C600000D0C4EAD4E0EDB7FEB7D283C1838BECC9
:102C700091E0948383830E945229809123060F90D0
:102C80000F900F900F9080FF22C000D000D0EDB7C2
:102C9000FEB7D283C18383EC91E0948383830E9447
:102CA00052298091310690913206845690400F90BF
:102CB0000F900F900F902091DE043091DF042817C1
:102CC00039070CF0D9C0809123068E7F21C000D037
:102CD00000D0EDB7FEB7D283C1838BEB91E0948334
:102CE00083830E94522980913106909132068C593B
:102CF0009F4F0F900F900F900F902091DE04309116
:102D0000DF04821793070CF0B7C08091230681601F
:102D100080932306B1C000D000D0C4EAD4E0EDB760
:102D2000FEB7D283C18381EB91E0948383830E94B9
:102D300052290F900F900F900F9080914A06882390
:102D400001F100D000D0EDB7FEB7D283C18387EA8E
:102D500091E0948383830E9452298091310690915F
:102D60003206845690400F900F900F900F90209154
:102D7000DE043091DF04281739071CF510924A064B
:102D800020C000D000D0EDB7FEB7D283C1838AE95E
:102D900091E0948383830E9452298091310690911F
:102DA00032068C599F4F0F900F900F900F902091EB
:102DB000DE043091DF04821793071CF481E08093D6
:102DC0004A068CE996E06BEF73E040914A060E9458
:102DD0001B3052C000D000D0A4EAEA2EA4E0FA2EA4
:102DE000EDB7FEB7F282E18289E891E094838383B4
:102DF0000E9452298DB79EB708970FB6F8949EBFD0
:102E00000FBE8DBF0DB71EB70F5F1F4FEDB7FEB7DB
:102E1000F282E18288EF91E0F801938382836091EE
:102E20004B0670E080E090E00E94353420E030E016
:102E300040E251E40E949C33F801648375838683E9
:102E4000978386E790E09187808780E290E0938780
:102E500082870E9463298DB79EB70C960FB6F894AF
:102E60009EBF0FBE8DBF80914B0690E060E873E07F
:102E70000E94D10C80934B0684EA94E00E942B05BB
:102E8000DF91CF911F910F91FF90EF9008952F92B6
:102E90003F924F925F926F927F928F929F92AF92EA
:102EA000BF92CF92DF92EF92FF920F931F93DF9327
:102EB000CF93CDB7DEB72B970FB6F894DEBF0FBE1A
:102EC000CDBF888769870E94FC3020915A063091D7
:102ED0005B0640915C0650915D0626173707480750
:102EE000590708F069C180915E068823C9F0809374
:102EF000AE0210925E0680E092E0909360068093AE
:102F00005F060E94FC306C507E4F8F4F9F4F609346
:102F10005A0670935B0680935C0690935D0607C12A
:102F20008091AE02282E33242091DA042F83009161
:102F30005F06109160063091C70439838091E704E1
:102F40008E83909151069D83E09014056090F40467
:102F50007090F5048090F6049090F70490914B06E1
:102F60004090AC025090AD0280915206A82FB0E084
:102F7000BC83AB83B0915306BA83F09013053B86B4
:102F80002A86A92EBB24CC24DD24EA85FB85319634
:102F9000FB87EA8737972CF021E030E03B872A87D0
:102FA0001CC08A859B858330910539F18430910559
:102FB0003CF48130910589F0029709F07FC015C07B
:102FC000AA85BB85A530B10509F44EC0A530B10571
:102FD00004F1169709F072C058C0BF81B23008F0F2
:102FE0006DC00DE012E081E070C0E981E33009F4CA
:102FF00065C00AE112E082E068C0FE81F23008F0AC
:103000005DC02D81222309F459C007E212E083E05C
:103010005CC031E03E1598F0C601B5010E94353420
:1030200020E030E040E251E40E949C339B01AC017F
:10303000C401B3010E94953388230CF03FC004E320
:1030400012E083E0E81649F094E0E91649F0A2E0C6
:10305000EA1641F401E412E005C00EE412E002C0F9
:103060000BE512E084E031C0EB81FC814E165F0677
:103070002CF5FDE94F16FFEF5F0601F12A812223AF
:10308000E9F408E612E085E020C03F813230B0F478
:1030900081E08F1598F493E0F91649F0A4E0FA1650
:1030A00049F0B2E0FB1651F405E712E005C001E873
:1030B00012E002C00EE812E086E007C0EA85FB8558
:1030C000E215F30509F061CF60C01093600600932C
:1030D0005F0680935E0681E0809354060E94FC3078
:1030E00068517C4F8F4F9F4F60935A0670935B06D9
:1030F00080935C0690935D060E94FC306056704F92
:103100008F4F9F4F609356067093570680935806D3
:103110009093590680915506882321F084EA94E023
:103120000E9494051092550602C01092540604EABB
:1031300014E0C801688549850E946F04C8010E9497
:10314000470500D000D000D0EDB7FEB73196ADB73F
:10315000BEB712961C930E9311978BE992E093835E
:10316000828380915F0690916006958384830E949C
:103170006329EDB7FEB736960FB6F894FEBF0FBEC3
:10318000EDBFC8010E942B0517C010936006009385
:103190005F0610925E060E94FC3020915606309128
:1031A0005706409158065091590626173707480789
:1031B000590708F4BACFBBCF2B960FB6F894DEBFF1
:1031C0000FBECDBFCF91DF911F910F91FF90EF9078
:1031D000DF90CF90BF90AF909F908F907F906F9037
:1031E0005F904F903F902F900895EF92FF920F9332
:1031F0001F9380916106843009F056C09091DB04E2
:10320000943008F027C180916A068917A1F1909344
:103210006A060E94FC30609366067093670680938E
:1032200068069093690690916A068091AF0298179C
:1032300011F580915506813091F0813018F082307F
:10324000B1F413C011E0109355060E94FC30615395
:1032500075478040904030F41093620608C082E0C9
:10326000809355061092620602C01092550684EAB9
:1032700094E00E9494050E94FC30209166063091F3
:1032800067064091680650916906621B730B840BB8
:10329000950B615D77408040904008F4DBC08091E1
:1032A000DB048093AF02D6C0853029F48091A4025C
:1032B0009091A50214C0863029F48091A6029091C5
:1032C000A7020DC0873029F48091A8029091A9022D
:1032D00006C0883041F48091AA029091AB0290938D
:1032E00065068093640680916306209164063091A0
:1032F0006506882309F04AC0C901895097408F5A52
:103300009440C8F40E94FC3061537547804090405F
:1033100020F481E0809362060CC0809162068823CD
:1033200041F480915406882321F484EA94E00E94B9
:10333000940582E028C044E0203B340768F4809183
:103340005506882349F01092620684EA94E00E94B0
:103350009405109255067EC0205B344029553240BA
:1033600008F078C080915506813009F473C08091CF
:103370005406882309F06EC01092620684EA94E035
:103380000E94940581E08093550664C0215B34401F
:1033900008F460C00E94FC30615375478040904043
:1033A00008F041C0809162068823E9F5E090660646
:1033B000F0906706009168061091690688EE93E028
:1033C000A0E0B0E0E80EF91E0A1F1B1F0E94FC30AF
:1033D000E616F70608071907E8F581E0809362060C
:1033E00017C01092620684EA94E00E9494058091CE
:1033F0005506823019F41092550603C08F5F8093F2
:10340000550680915506823018F082E0809355066B
:103410000E94FC306093660670936706809368068E
:103420009093690617C0E0906606F09067060091D9
:1034300068061091690688EE93E0A0E0B0E0E80E1F
:10344000F91E0A1F1B1F0E94FC30E616F70608072C
:10345000190738F21F910F91FF90EF900895809116
:103460006106843010F00E94F5188091620688236E
:1034700019F00E94A01508958091070480FF08C0EC
:1034800060916D0480916B0490E070E00E9447179A
:1034900080915506823008F0FDC1A82FB0E0FD01F3
:1034A000EF5FFB4F808185FF0BC0FD01E35EFB4FAB
:1034B0006081A55EBB4F8C9190E070E00E940D157D
:1034C00080915506A82FB0E0FD01EF5FFB4F808192
:1034D00086FF0BC0FD01EF5DFB4F6081A15EBB4F1E
:1034E0008C9190E070E00E94CE1480915106882368
:1034F00009F43FC080915506A82FB0E0FD01EF5FB1
:10350000FB4F808187FF0BC0FD01EB5DFB4F6081AE
:10351000AD5DBB4F8C9190E070E00E947C14809177
:103520005506A82FB0E0FD01ED5FFB4F808184FFC1
:103530000BC0FD01E35CFB4F6081A55CBB4F8C9130
:1035400090E070E00E94231480915506A82FB0E00F
:10355000FD01ED5FFB4F808183FF0BC0FD01E75C48
:10356000FB4F6081A95CBB4F8C9190E070E00E94A2
:103570000C1480915506A82FB0E0FD01EB5FFB4FC6
:10358000808187FF0BC0FD01EB5AFB4F6081AD5A74
:10359000BB4F8C9190E070E00E94B3138091550670
:1035A000A82FB0E0FD01E95FFB4F808183FF0BC0D6
:1035B000FD01EB58FB4F6081AD58BB4F8C9190E003
:1035C00070E00E941E1280915106882309F444C0C5
:1035D0008091E704823008F43FC080915506A82FFF
:1035E000B0E0FD01E75FFB4F808182FF0BC0FD0172
:1035F000EF57FB4F6081A158BB4F8C9190E070E07A
:103600000E94641280915506A82FB0E0FD01EB5F87
:10361000FB4F808182FF0BC0FD01EF5AFB4F6081A1
:10362000A15BBB4F8C9190E070E00E945C13809195
:103630005506A82FB0E0FD01EB5FFB4F808183FFB3
:103640000BC0FD01E75AFB4F6081A95ABB4F8C911B
:1036500090E070E00E94051380915506A82FB0E01D
:10366000FD01ED5FFB4F808181FF0BC0FD01EF5C31
:10367000FB4F6081A15DBB4F8C9190E070E00E9498
:10368000DC1180915506A82FB0E0FD01ED5FFB4FE6
:10369000808180FF0BC0FD01E35DFB4F6081A55D74
:1036A000BB4F8C9190E070E00E949A11809155067A
:1036B000A82FB0E0FD01E95FFB4F808186FF0BC0C2
:1036C000FD01E358FB4F6081A558BB4F8C9190E002
:1036D00070E00E945A1180915506A82FB0E0FD01BC
:1036E000EF5FFB4F808182FF0BC0FD01EB5EFB4F64
:1036F0006081AD5EBB4F8C9190E070E00E941A112A
:1037000080915506A82FB0E0FD01EF5FFB4F80814F
:1037100081FF0BC0FD01EF5EFB4F6081A15FBB4FDE
:103720008C9190E070E00E94DA1080915506A82FED
:10373000B0E0FD01EB5FFB4F808184FF0BC0FD011A
:10374000EF59FB4F6081A15ABB4F8C9190E070E024
:103750000E949A1080915506A82FB0E0FD01EB5F02
:10376000FB4F808185FF0BC0FD01EB59FB4F608152
:10377000AD59BB4F8C9190E070E00E940210809197
:103780005506A82FB0E0FD01EF5FFB4F808183FF5E
:103790000BC0FD01E75EFB4F6081A95EBB4F8C91C2
:1037A00090E070E00E94BC0F80915506A82FB0E019
:1037B000FD01EB5FFB4F808180FF0BC0FD01E35BF0
:1037C000FB4F6081A55BBB4F8C9190E070E00E9445
:1037D000670F80915506A82FB0E0FD01EF5FFB4F0A
:1037E000808184FF0BC0FD01E75DFB4F6081A95D17
:1037F000BB4F8C9190E070E00E94270F809155069E
:10380000A82FB0E0FD01E75FFB4F808181FF18C06A
:1038100080914A06FD01ED57FB4F813049F4AB57CB
:10382000BB4F6C91808190E070E00E940B0E08C04D
:10383000AB57BB4F6C91808190E070E00E945E0EB0
:1038400080915506A82FB0E0FD01ED5FFB4F808110
:1038500087FF0BC0FD01E75BFB4F6081A95BBB4F9E
:103860008C9190E070E00E94880D80915506A82F01
:10387000B0E0FD01EB5FFB4F808186FF0BC0FD01D7
:10388000E759FB4F6081A959BB4F8C9190E070E0E4
:103890000E942D0D089584EA94E00E9494050E94F0
:1038A00047150E94060A0895CF93DF93EC0184EA3E
:1038B00094E00E946B04C817D9073CF084EA94E0B6
:1038C0000E946004892B09F42397CE01DF91CF91E8
:1038D0000895EF92FF920F931F93CF93DF93009180
:1038E000550610E08AEF90E0089F7001099FF00CE8
:1038F000189FF00C1124C7010E94EB0AF801EF5F3A
:10390000FB4F882319F08081816002C080818E7F07
:10391000808380915506C82FD0E0C70102960E948F
:10392000EB0AC55FDB4F888380915506C82FD0E036
:10393000C70104960E94EB0A90E00E94541CC35FEA
:10394000DB4F88830091550610E0C70188569F4FD2
:103950000E94EB0AF801EF5FFB4F882319F080818A
:10396000806102C080818F7E808380915506C82F40
:10397000D0E0C70186569F4F0E94EB0AC95DDB4F1E
:10398000888380915506C82FD0E0C70184569F4F89
:103990000E94EB0A90E00E94541CC75DDB4F8883B5
:1039A0000091550610E0C70106960E94EB0AF80147
:1039B000EF5FFB4F882319F08081826002C0808115
:1039C0008D7F808380915506C82FD0E0C70108966F
:1039D0000E94EB0AC15FDB4F888380915506C82F98
:1039E000D0E0C7010A960E94EB0A90E00E94541CA6
:1039F000CF5EDB4F88830091550610E0C7010C961F
:103A00000E94EB0AF801EF5FFB4F882319F08081D9
:103A1000846002C080818B7F808380915506C82F8F
:103A2000D0E0C7010E960E94EB0ACD5EDB4F888383
:103A300080915506C82FD0E0C70140960E94EB0A3E
:103A400090E00E94541CCB5EDB4F888300915506AA
:103A500010E0C70142960E94EB0AF801EF5FFB4FAE
:103A6000882319F08081886002C08081877F8083ED
:103A700080915506C82FD0E0C70144960E94EB0AFA
:103A8000C95EDB4F888380915506C82FD0E0C701FF
:103A900046960E94EB0A90E00E94541CC75EDB4FE2
:103AA00088830091550610E0C7014E960E94EB0AEC
:103AB000F801EF5FFB4F882319F08081806202C01C
:103AC00080818F7D808380915506C82FD0E0C7010B
:103AD00080960E94EB0AC55EDB4F88838091550675
:103AE000C82FD0E0C70182960E94EB0A90E00E94A6
:103AF000541CC35EDB4F88830091550610E0C7015C
:103B000084960E94EB0AF801EF5FFB4F882319F0BF
:103B10008081806402C080818F7B80838091550684
:103B2000C82FD0E0C70186960E94EB0AC15EDB4F2A
:103B3000888380915506C82FD0E0C70188960E94DF
:103B4000EB0A90E00E94541CCF5DDB4F888300910C
:103B5000550610E0C7018A960E94EB0AF801EF5F54
:103B6000FB4F882319F08081806802C080818F77A5
:103B7000808380915506C82FD0E0C7018C960E94A3
:103B8000EB0ACD5DDB4F888380915506C82FD0E0CE
:103B9000C7018E960E94EB0A90E00E94541CCB5DF8
:103BA000DB4F88830091550610E0C701C0960E9444
:103BB000EB0AF801ED5FFB4F882319F080818160EB
:103BC00002C080818E7F808380915506C82FD0E00F
:103BD000C701C2960E94EB0AC55DDB4F88838091C6
:103BE0005506C82FD0E0C701C4960E94EB0A90E0AA
:103BF0000E94541CC35DDB4F88830091550610E082
:103C0000C701C6960E94EB0AF801ED5FFB4F8823BF
:103C100019F08081826002C080818D7F80838091D5
:103C20005506C82FD0E0C701C8960E94EB0AC15DB7
:103C3000DB4F888380915506C82FD0E0C701CA9614
:103C40000E94EB0A90E00E94541CCF5CDB4F8883FB
:103C50000091550610E0C701CC960E94EB0AF801CE
:103C6000ED5FFB4F882319F08081846002C0808162
:103C70008B7F808380915506C82FD0E0C701CE96F8
:103C80000E94EB0ACD5CDB4F888380915506C82FDC
:103C9000D0E0C701805C9F4F0E94EB0A90E00E9439
:103CA000541CCB5CDB4F88830091550610E0C701A4
:103CB000885B9F4F0E94EB0AF801ED5FFB4F882362
:103CC00019F08081806102C080818F7E8083809125
:103CD0005506C82FD0E0C701865B9F4F0E94EB0AB4
:103CE000C55CDB4F888380915506C82FD0E0C701A3
:103CF000845B9F4F0E94EB0A90E00E94541CC35CBF
:103D0000DB4F88830091550610E0C7018E5B9F4F03
:103D10000E94EB0AF801ED5FFB4F882319F08081C8
:103D2000886002C08081877F808380915506C82F7C
:103D3000D0E0C7018C5B9F4F0E94EB0AC95CDB4F50
:103D4000888380915506C82FD0E0C7018A5B9F4FBA
:103D50000E94EB0A90E00E94541CC75CDB4F8883F2
:103D60000091550610E0C701805B9F4F0E94EB0A4F
:103D7000F801ED5FFB4F882319F08081806202C05B
:103D800080818F7D808380915506C82FD0E0C70148
:103D90008E5A9F4F0E94EB0AC15CDB4F8883809153
:103DA0005506C82FD0E0C7018C5A9F4F0E94EB0ADE
:103DB00090E00E94541CCF5BDB4F88830091550636
:103DC00010E0C7018A5A9F4F0E94EB0AF801ED5F8D
:103DD000FB4F882319F08081806402C080818F7B33
:103DE000808380915506C82FD0E0C701885A9F4F25
:103DF0000E94EB0ACD5BDB4F888380915506C82F6C
:103E0000D0E0C701865A9F4F0E94EB0A90E00E94C3
:103E1000541CCB5BDB4F88830091550610E0C70133
:103E200082569F4F0E94EB0AF801ED5FFB4F8823FB
:103E300019F08081806802C080818F7780838091B3
:103E40005506C82FD0E0C70180569F4F0E94EB0A4D
:103E5000C95BDB4F888380915506C82FD0E0C7012E
:103E60008E559F4F0E94EB0A90E00E94541CC75B46
:103E7000DB4F88830091550610E0C7018E599F4F94
:103E80000E94EB0AF801EB5FFB4F882319F0808159
:103E9000816002C080818E7F808380915506C82F0B
:103EA000D0E0C7018C599F4F0E94EB0AC55BDB4FE6
:103EB000888380915506C82FD0E0C7018A599F4F4B
:103EC0000E94EB0A90E00E94541CC35BDB4F888386
:103ED0000091550610E0C70182599F4F0E94EB0ADE
:103EE000F801EB5FFB4F882319F08081846002C0EA
:103EF00080818B7F808380915506C82FD0E0C701D9
:103F000080599F4F0E94EB0AC15BDB4F88838091F1
:103F10005506C82FD0E0C7018E589F4F0E94EB0A6C
:103F200090E00E94541CCF5ADB4F888300915506C5
:103F300010E0C70184579F4F0E94EB0AF801EB5F26
:103F4000FB4F882319F08081806802C080818F77C1
:103F5000808380915506C82FD0E0C70182579F4FBC
:103F60000E94EB0ACD5ADB4F888380915506C82FFB
:103F7000D0E0C70180579F4F0E94EB0A90E00E945B
:103F8000541CCB5ADB4F88830091550610E0C701C3
:103F90008E569F4F0E94EB0AF801EB5FFB4F882380
:103FA00019F08081826002C080818D7F8083809142
:103FB0005506C82FD0E0C7018C569F4F0E94EB0AD0
:103FC000C55ADB4F888380915506C82FD0E0C701C2
:103FD0008A569F4F0E94EB0A90E00E94541CC35ADD
:103FE000DB4F88830091550610E0C7018C589F4F26
:103FF0000E94EB0AF801EB5FFB4F882319F08081E8
:10400000886002C08081877F808380915506C82F99
:10401000D0E0C7018A589F4F0E94EB0AC95ADB4F74
:10402000888380915506C82FD0E0C70188589F4FDC
:104030000E94EB0A90E00E94541CC75ADB4F888311
:104040000091550610E0C70186589F4F0E94EB0A69
:10405000F801EB5FFB4F882319F08081806102C07B
:1040600080818F7E808380915506C82FD0E0C70164
:1040700084589F4F0E94EB0AC15ADB4F888380917E
:104080005506C82FD0E0C70182589F4F0E94EB0A07
:1040900090E00E94541CCF59DB4F88830091550655
:1040A00010E0C70180589F4F0E94EB0AF801EB5FB8
:1040B000FB4F882319F08081806202C080818F7D50
:1040C000808380915506C82FD0E0C7018E579F4F3F
:1040D0000E94EB0ACD59DB4F888380915506C82F8B
:1040E000D0E0C7018C579F4F0E94EB0A90E00E94DE
:1040F000541CCB59DB4F88830091550610E0C70153
:104100008A579F4F0E94EB0AF801EB5FFB4F882311
:1041100019F08081806402C080818F7B80838091D0
:104120005506C82FD0E0C70188579F4F0E94EB0A61
:10413000C959DB4F888380915506C82FD0E0C7014D
:1041400086579F4F0E94EB0A90E00E94541CC7596B
:10415000DB4F88830091550610E0C7018C559F4FB7
:104160000E94EB0AF801E95FFB4F882319F0808178
:10417000816002C080818E7F808380915506C82F28
:10418000D0E0C7018A559F4F0E94EB0AC559DB4F0B
:10419000888380915506C82FD0E0C70188559F4F6E
:1041A0000E94EB0A90E00E94541CC359DB4F8883A5
:1041B0000091550610E0C70180559F4F0E94EB0A01
:1041C000F801E95FFB4F882319F08081846002C009
:1041D00080818B7F808380915506C82FD0E0C701F6
:1041E0008E549F4F0E94EB0AC159DB4F8883809108
:1041F0005506C82FD0E0C7018C549F4F0E94EB0A90
:1042000090E00E94541CCF58DB4F888300915506E4
:1042100010E0C7018A549F4F0E94EB0AF801E95F42
:10422000FB4F882319F08081886002C08081877FDE
:10423000808380915506C82FD0E0C70188549F4FD6
:104240000E94EB0ACD58DB4F888380915506C82F1A
:10425000D0E0C70186549F4F0E94EB0A90E00E9475
:10426000541CCB58DB4F88830091550610E0C701E2
:1042700084549F4F0E94EB0AF801E95FFB4F8823AB
:1042800019F08081806102C080818F7E808380915F
:104290005506C82FD0E0C70182549F4F0E94EB0AF9
:1042A000C958DB4F888380915506C82FD0E0C701DD
:1042B00080549F4F0E94EB0A90E00E94541CC75804
:1042C000DB4F88830091550610E0C701845A9F4F49
:1042D0000E94EB0AF801E95FFB4F882319F0808107
:1042E000806402C080818F7B808380915506C82FB7
:1042F000D0E0C701825A9F4F0E94EB0AC558DB4F9E
:10430000888380915506C82FD0E0C701805A9F4FFF
:104310000E94EB0A90E00E94541CC358DB4F888334
:104320000091550610E0C70180529F4F0E94EB0A92
:10433000F801E75FFB4F882319F08081846002C099
:1043400080818B7F808380915506C82FD0E0C70184
:104350008E519F4F0E94EB0AC158DB4F888380919A
:104360005506C82FD0E0C7018C519F4F0E94EB0A21
:1043700090E00E94541CCF57DB4F88830091550674
:1043800010E0C7018C529F4F0E94EB0AF801E75FD3
:10439000FB4F882319F08081826002C080818D7F6D
:1043A000808380915506C82FD0E0C7018A529F4F65
:1043B0000E94EB0ACD57DB4F888380915506C82FAA
:1043C000D0E0C70188529F4F0E94EB0A90E00E9404
:1043D000541CCB57DB4F8883DF91CF911F910F91F6
:1043E000FF90EF9008954F925F927F928F929F92ED
:1043F000AF92BF92CF92DF92EF92FF920F931F93F3
:10440000DF93CF93CDB7DEB7C854D0400FB6F89442
:10441000DEBF0FBECDBF04EA14E0C8010E949405C0
:10442000C80166E049E00E946F04C8010E94470588
:1044300000D000D0EDB7FEB7128301838FEF91E07B
:10444000948383830E9452290F900F900F900F90B6
:10445000C8010E942B0500D000D007E814E0EDB79A
:10446000FEB7128301838FEE91E0948383830E94D1
:10447000522944EE442E41E0542EEE24FF24CC2455
:10448000DD240F900F900F900F90702E012F39E0C8
:10449000A32EB12CAC0EBD1E4E010894811C911CA4
:1044A00087E894E00E94062A982F8D3031F08D30F5
:1044B000DCF180538230C0F530C01830A1F599810D
:1044C000892F8053823078F5913311F490E801C040
:1044D00090E08A81813309F4905C8B81813309F407
:1044E000905E8C81813309F4905F8D81813309F472
:1044F000985F8E81813309F49C5F8F81813309F449
:104500009E5F8885813309F49F5FF501EE0DFF1DE5
:1045100090830894E11CF11C06C0F401E10FF11D29
:1045200090831F5F01C010E0F0E4EF16F104C9F4BE
:1045300084EA94E0B601A5010E947F040894C11C9E
:10454000D11C00D000D0EDB7FEB771820283548237
:1045500043820E945229EE24FF240F900F900F9067
:104560000F90FFEFCF16D10409F00CF499CFC85B80
:10457000DF4F0FB6F894DEBF0FBECDBFCF91DF91F6
:104580001F910F91FF90EF90DF90CF90BF90AF9071
:104590009F908F907F905F904F900895DF92EF9261
:1045A000FF920F931F93DF93CF93CDB7DEB72A9778
:1045B0000FB6F894DEBF0FBECDBF63E0E62EF12C40
:1045C000EC0EFD1E53E0D52EF6C30E94FC30605267
:1045D0007E4480409040C8F40E94FC30695873418A
:1045E0008040904090F01A3011F01D3031F48091ED
:1045F0001F068F5F80931F0602C010921F068091D6
:104600001F06833011F40E94F321812F65E175E0CC
:104610000E94F106882311F400E0C7C380911905B8
:1046200090911A05A0911B05B0911C05863E46EAA3
:10463000940746E2A4074DE7B40709F48EC2873E0B
:1046400056EA950756E2A5075DE7B50708F0EFC003
:104650008832EEE59E07E2EDAE07E4E2BE0709F41C
:1046600027C28932FEE59F07F2EDAF07F4E2BF07EC
:1046700008F06AC088392CE292072AE1A20726E1F5
:10468000B20709F41EC289393CE293073AE1A30755
:1046900036E1B30740F586314AEA940747E3A407B9
:1046A0004BE0B40709F404C287315AEA950757E38F
:1046B000A5075BE0B50738F48E5F9B4CA74CB9406B
:1046C00009F069C360C38430FAE99F07F7EDAF07CB
:1046D000FEE0BF0709F4ECC18259934AAC4EB441E5
:1046E00009F059C3E5C184373BEE93073AE7A307C6
:1046F0003BE1B30709F4DCC185374BEE94074AE789
:10470000A4074BE1B40780F480355FED95075DEEBB
:10471000A50758E1B50709F40BC38E5C9844A7457B
:10472000BA4109F038C319C28434FBED9F07F0E7A2
:10473000AF07FDE1BF0709F426C3825D924CA24892
:10474000BE4109F028C3BDC1883536EB93073DEF64
:10475000A3073AE4B30709F4CDC2893546EB9407C1
:104760004DEFA4074AE4B40788F5863E55ED95075A
:104770005AEDA50753E3B50709F448C1873EE5EDB7
:104780009E07EAEDAE07E3E3BE0780F48E37F9EA51
:104790009F07FBE5AF07F6E2BF0709F492C1825518
:1047A0009342A649B64209F0F6C254C2883F3CEA99
:1047B00093073EEEA30734E3B30709F4E4C2865A35
:1047C0009E40A241B84409F0E6C27DC280365BED4E
:1047D00095075BE3A5075EE6B50709F469C1813675
:1047E000EBED9E07EBE3AE07EEE6BE0780F4823EFC
:1047F000F5E59F07FCE9AF07F6E6BF0709F48AC2B3
:104800008C5E9943A647BB4609F0C5C2BCC28A3B31
:1048100037EC930731E2A30734E7B30709F4F6C096
:104820008A57974CA94DBB4709F0B5C2ACC28A3B29
:1048300054E8950755E2A5075EEBB50709F46AC28F
:104840008B3BE4E89E07E5E2AE07EEEBBE0708F01F
:104850006AC08E37F2E19F07FAE6AF07FBE9BF07B0
:1048600009F426C18F3722E192072AE6A2072BE935
:10487000B20740F582353AEE930730E8A3073AE8ED
:10488000B30709F415C183354AEE940740E8A4073D
:104890004AE8B40738F486549340A24CB54809F06E
:1048A0007AC271C28C38E5E89E07E7EAAE07E8E90C
:1048B000BE0709F452C18A569E42A246B94909F080
:1048C0006AC201C280322EE4920729EAA20721EBD4
:1048D000B20709F41FC281323EE4930739EAA30705
:1048E00031EBB30780F48A3746EF940741EFA40712
:1048F0004DE9B40709F431C18E5F964BA942B54A20
:1049000009F049C22AC18A38E7EF9E07E7ECAE07F3
:10491000E8EBBE0709F4D5C0845A9040AB49BA4BC6
:1049200009F039C230C2843629ED920720EEA20781
:1049300027EDB20709F46AC0853639ED930730EEEA
:10494000A30737EDB30788F586384BE3940740EAB1
:10495000A40744ECB40709F4DDC187385BE395078D
:1049600050EAA50754ECB50780F48C36E8E69E07BC
:10497000E3E4AE07E2ECBE0709F45CC1805894475B
:10498000A041B44C09F007C29CC084352DE29207C7
:104990002FEFA20725ECB20709F48AC08659954388
:1049A000A840B24D09F0F7C155C18E344DE59407CA
:1049B0004EE3A40743EEB40709F47AC08F345DE5F3
:1049C00095075EE3A50753EEB50780F48437E7E368
:1049D0009E07E4EDAE07EEEDBE0709F49BC1865BD2
:1049E0009342A34AB24E09F0D6C1B7C0823920E73C
:1049F000920726E8A2072BEFB20709F4C4C1825F31
:104A00009D4EA442BD4F09F0C6C18DC10E94FC302D
:104A10006093C8047093C9048093CA049093CB0434
:104A2000D092C70485E195E060E170E00E94C5087E
:104A30000E9404347093CD046093CC0485E195E02A
:104A400064E170E00E94C5080E9404347093CF04B2
:104A50006093CE0485E195E068E170E00E94C508AE
:104A60000E9404348B017093D1046093D004609150
:104A7000D2047091D3048091D4049091D50420E0A5
:104A800030E040E050E00E949533882379F4B8018B
:104A9000882777FD8095982F0E9437346093D6043D
:104AA0007093D7048093D8049093D90401E074C123
:104AB00080911F058093DA04809120058093DB04A8
:104AC0006AC185E195E060E070E00E94C50820E0E1
:104AD00030E048EC52E40E946A350E94043470933E
:104AE000DD046093DC04693C710520F01092DD0464
:104AF0001092DC048091390590913A059093DF047F
:104B00008093DE0480913B0590913C059093E104F5
:104B10008093E00480913F05909140059093A50219
:104B20008093A40280914305909144059093A7023D
:104B30008093A60280914505909146059093A90225
:104B40008093A80280914705909148059A838983B4
:104B50009093AB028093AA021EC160911F057091D1
:104B6000200580912105909122050E94373420E88C
:104B700036E948E15BE40E949C336093D204709371
:104B8000D3048093D4049093D5046091230570914D
:104B900024058091250590912605D7016C931196E7
:104BA0007C93119712968C93129713969C930E9464
:104BB000373420E836E948E15BE40E949C33609397
:104BC000E2047093E3048093E4049093E5048091FD
:104BD00044058093E604809143058093E70485E1D2
:104BE00095E060E170E00E94C5086093D604709380
:104BF000D7048093D8049093D90485E195E068E0C8
:104C000070E00E94C5086093E8047093E904809303
:104C1000EA049093EB0485E195E064E170E00E9482
:104C2000C5086093EC047093ED048093EE049093B8
:104C3000EF04B1C085E195E068E070E00E94C5082E
:104C400090586093F0047093F1048093F204909371
:104C5000F304A1C085E195E060E070E00E94C50822
:104C60006093F4047093F5048093F6049093F70432
:104C700085E195E064E070E00E94C50820E030E046
:104C800048EC52E40E946A350E9404347093F9049F
:104C90006093F80485E195E064E170E00E94C50846
:104CA0000E9404347093FB046093FA0485E195E05C
:104CB00068E170E00E94C5080E9404347093FD040E
:104CC0006093FC0468C085E195E064E070E00E94B8
:104CD000C5080E940434882777FD8095982F0E948C
:104CE00037346093FE047093FF0480930005909323
:104CF000010551C085E195E068E070E00E94C508BB
:104D00000E940434709561957F4F70930305609302
:104D1000020541C080917F05809304058091800544
:104D20008093050538C080911F058093060533C028
:104D300085E195E060E070E00E94C508609307059A
:104D4000709308058093090590930A0585E195E025
:104D500064E070E00E94C50860930B0570930C0539
:104D600080930D0590930E0585E195E068E070E075
:104D70000E94C50860930F0570931005809311057C
:104D80009093120508C080912B05809313058091A4
:104D900030058093140500E080911605823229F4D5
:104DA00085E195E063E20E94DD098EEB90E00E94D0
:104DB0006331002331F587E894E00E94D629181664
:104DC0001906F4F487E894E00E94062A182F8091CF
:104DD000C704882309F019CCF8CB1092C70401E06E
:104DE000802F90E02A960FB6F894DEBF0FBECDBF9D
:104DF000CF91DF911F910F91FF90EF90DF90089579
:104E000000E02091C8043091C9044091CA04509137
:104E1000CB04205F384D4F4F5F4F2F833887498732
:104E20005A870E94FC302F81388549855A8526177C
:104E300037074807590788F2D3CF1F93CF93DF93E3
:104E400085E090E06CE070E00E947D1568EE73E014
:104E500080E090E00E940A3187E894E00E94532AA3
:104E6000C0E0D0E010E0CE016DE171E00E94A43618
:104E7000892BA9F41F5E84EA94E0612F4CE00E9424
:104E80006F0484EA94E00E94470584EA94E06EEEA1
:104E90000E94770584EA94E00E942B05105161E09E
:104EA00070E080E090E00E940A31219687E0C13DE9
:104EB000D807C9F6DF91CF911F91089586E061E090
:104EC0000E94413208950F931F9386E061E00E9493
:104ED000023207E814E0C80140E051EE60E070E003
:104EE0000E94742910939E0600939D060E945E27DF
:104EF00084EA94E00E94CD050E944B1C64EF71E0AF
:104F000080E090E00E940A3183EF93E00E94EB0A78
:104F1000813011F00E94FC0C0E945C0A1092550630
:104F200007C00E94691C809155068F5F80935506CB
:104F3000809155068230A8F3109255060E941D27D5
:104F400086EB94E062E379E224E630E040E050E072
:104F500000E00E94273084EA94E00E94940586EBEA
:104F600094E00E948D301F910F9108952F923F92EF
:104F70004F925F926F927F928F929F92AF92BF9269
:104F8000CF92DF92EF92FF920F931F93DF93CF9315
:104F900000D000D0CDB7DEB780915106882309F448
:104FA000E1C0E0907606F0907706009178061091C7
:104FB0007906C801B7019F7725E33AEF4EE85CE335
:104FC0000E946A350E94993369837A838B839C831C
:104FD000C801B7012091D2043091D3044091D40488
:104FE0005091D5040E94CE321B012C019F7720ECFA
:104FF0003BE649ED57E40E946A355B016C01609124
:105000007A0670917B0680917C0690917D062091B6
:10501000E2043091E3044091E4045091E5040E94DD
:10502000CE323B014C019F7720EC3BE649ED57E443
:105030000E946A3529813A814B815C810E946A35E0
:105040007B018C01C601B501A60195010E946A355C
:105050005B016C01C801B701A80197010E946A3584
:105060009B01AC01C601B5010E94CF320E94F1350F
:105070000E9404346093440670934506809346066C
:105080009093470660E070E080E89FE329813A81D1
:105090004B815C810E949C339B01AC01C201B10138
:1050A0000E946A3597FA909497F89094A40193011E
:1050B0000E94423320EE3EE245E652E40E946A3509
:1050C00020E030E044EB52E40E94CF320E940434EE
:1050D0009B01AC0197FF04C028593E4F4F4F5F4FD3
:1050E000CA01B901645B70408040904097FF06C0E0
:1050F000CA01B9016C547F4F8F4F9F4F0E943734C4
:105100002091D6043091D7044091D8045091D9040D
:105110000E94CE320E94043497FF04C068597E4F2B
:105120008F4F9F4F0E94373420E030E044EB53E430
:105130000E949C3320E030E040E851E40E946A3550
:105140000E94CD3520E030E040E85FE30E94CF329E
:105150000E94093460934306613108F46CC01092D8
:10516000430669C08091E704823008F464C08091EE
:10517000E604853008F45FC0A0907E068DE18A15B4
:1051800008F459C0E090E804F090E9040091EA04C2
:105190001091EB0460917F067091800680918106EA
:1051A00090918206A80197010E94CE329F7720E05D
:1051B00030E040E05FE30E945F3518165CF4109227
:1051C0007E06E0927F06F09280060093810610939F
:1051D000820631C08A2D8F5F80937E068E3159F50D
:1051E0008091D2049091D304A091D404B091D504BD
:1051F0008093760690937706A0937806B09379060D
:105200008091E2049091E304A091E404B091E5045C
:1052100080937A0690937B06A0937C06B0937D06DC
:10522000E0928306F092840600938506109386062A
:1052300081E0809351060F900F900F900F90CF91C7
:10524000DF911F910F91FF90EF90DF90CF90BF9073
:10525000AF909F908F907F906F905F904F903F9016
:105260002F900895809106058093AC021092AD02B4
:105270000E944E080E94F10A84EA94E00E94B62738
:105280000E942F1A08950E94CE22892B19F00E94A5
:105290003229089586EB94E00E94753008958FEFCF
:1052A0009FE70895DF93CF93CDB7DEB7FE01399620
:1052B0008D819E8161E04F8158859F010E94F32B73
:1052C000CF91DF910895DF93CF93CDB7DEB7FE0185
:1052D00039968D819E8160E04F8158859F010E94A3
:1052E000F32BCF91DF9108950F931F93DC01ED9184
:1052F000FC910288F389E02D20E030E000E010E02E
:1053000009951F910F9108958F92AF92CF92EF92CE
:10531000FF920F931F93DF93CF93CDB7DEB7FC01BE
:105320001382128288EE93E0A0E0B0E0848395833C
:10533000A683B7838AEE93E0918380835587448761
:1053400037872687118B008BF38AE28AC48AA58A65
:10535000868A70E0CB0123E0880F991F2A95E1F738
:105360009C012557394F308F278B8D56994F928F3F
:10537000818F81E090E002C0880F991F6A95E2F763
:1053800020919B06282B20939B06CF0140E051EEF5
:1053900060E070E00E947429CF91DF911F910F911E
:1053A000FF90EF90CF90AF908F900895FC01838D88
:1053B000882319F42FEF3FEF0DC00788F08DE02D03
:1053C0002081318182819381281B390B84819581D1
:1053D00028233923C9010895FC01838D882319F4FA
:1053E0002FEF3FEF11C0018CF28DE02D2081318134
:1053F00082819381281B390B20953095848195817A
:10540000282339232F5F3F4FC9010895FC01838D65
:10541000882361F0A789B08D2D913C911197129648
:105420008D919C9113972817390721F44FEF5FEF67
:10543000CA01089512968D919C9113971696ED913D
:10544000FC911797E80FF91F408112968D919C915E
:105450001397019614962D913C91159782239323CF
:1054600013969C938E93129750E0E2CFFC01838DAC
:10547000882351F00788F08DE02D208131818281D1
:1054800093812817390721F42FEF3FEFC9010895C1
:10549000828193810680F781E02DE80FF91F8081DA
:1054A000282F30E0F3CFDC015796ED91FC9158970F
:1054B00082819381918380835996ED91FC915A97D3
:1054C00080819181938382830895DC015B968C9126
:1054D0005B978823A9F15996ED91FC915A97208109
:1054E00031812F5F3F4F84819581282339235C963A
:1054F0008C915C97882329F0828193812817390742
:10550000F9F08281938128173907D9F3808191813D
:105510000680F781E02DE80FF91F60835996ED9121
:10552000FC915A97318320835296ED91FC915397C9
:10553000808156969C91892B808321E030E002C0C7
:1055400020E030E0C9010895CF93DF93EC011B8286
:105550001A828A819B81998388831D821C828E8115
:105560009F81009721F00E94C1031F821E82DF915C
:10557000CF9108950F931F938C01DC015296ED910A
:10558000FC915397208156968C91569755969C91F5
:105590005597892B80958223808357968D919C9176
:1055A00058970E94A42AF801818D928D0E94A42A06
:1055B000D8015B961C921F910F9108950F931F9332
:1055C000CF93DF938C01FC0113821282828193813D
:1055D0009183808341E0A1E0B0E001C04F5FFD0115
:1055E000042E02C0EE0FFF1F0A94E2F79B0182E037
:1055F0006130780710F020E032E0E217F30770F333
:10560000C1E0D0E002C0CC0FDD1F4A95E2F7219740
:10561000F801268137812115310541F0848195817A
:105620008C179D0789F0C9010E94C103F801D58339
:10563000C483CE0101960E9417039C01F801978351
:10564000868380E0232B09F081E0DF91CF911F91C9
:105650000F910895AF92BF92CF92DF92EF92FF9297
:105660000F931F93CF93DF937C015A016B01E901E4
:10567000DC015B968C915B978823F1F02115310555
:1056800039F45796ED91FC915897C481D5812196B4
:105690000115110549F4D7015996ED91FC915A97DE
:1056A000048115810F5F1F4FD701ED91FC91008898
:1056B000F189E02DC7010995F7018789908D209721
:1056C00011F4C0E8D0E0BE010E94DE2A882381F0F8
:1056D000D70159968D919C915A970115110511F496
:1056E00000E110E0B8010E94DE2A882309F04DC0D5
:1056F000D701ED91FC910088F189E02DC701099552
:1057000067C0D7015096ED91FC915197B0E0AB1670
:10571000B1EEBB06B0E0CB06B0E0DB0609F454C046
:1057200081E090E0D70154960C9002C0880F991F39
:105730000A94E2F7808360E079E08DE390E0A601CF
:1057400095010E94D9362150304040405040CA0156
:10575000B90122E030E040E050E00E94D936D701A4
:105760001C96ED91FC911D9730831E96ED91FC9156
:105770001F972083D7015296ED91FC91539780811A
:1057800055969C91892B808323C0D7015996ED9122
:10579000FC915A9713821282828193819183808334
:1057A0005796ED91FC9158971382128282819381D2
:1057B0009183808381E05B968C931A141B041C04F4
:1057C0001D040CF49ECFD6CF108220E130E0C7CF6D
:1057D000DF91CF911F910F91FF90EF90DF90CF90CD
:1057E000BF90AF9008952F923F924F925F926F9229
:1057F0007F928F929F92AF92BF92CF92DF92EF9261
:10580000FF920F931F93DF93CF93CDB7DEB76497CB
:105810000FB6F894DEBF0FBECDBF3C01688B5A8B2C
:10582000498B69011C01AE014F5F5F4F5C8B4B8B55
:10583000E989FA89488940FD659140FF6191FA8BB9
:10584000E98B662309F4D7C3653249F440FD85919D
:1058500040FF8191FA8BE98B8532B1F40CC06A303C
:1058600051F4D301ED91FC910190F081E02DC10143
:105870006DE009956AE0D301ED91FC910190F08112
:10588000E02DC1010995D4CF982F10E088249924E8
:105890001032B0F49B3269F09C3228F4903251F00F
:1058A000933271F40BC09D3239F0903349F411609A
:1058B00028C01260146025C0186023C0106121C088
:1058C00017FD2BC0892F80538A3078F416FF06C04D
:1058D000BAE09B9E902C1124980E13C0EAE08E9E95
:1058E000802C1124880E10620CC09E3221F416FD0B
:1058F00082C3106406C09C3611F4106802C098364A
:1059000061F4E989FA89488940FD959140FF9191B8
:10591000FA8BE98B992309F0BBCF892F855483300B
:1059200020F4812F8061905E07C0892F85568330D7
:1059300008F0E6C1812F8F7E86FD02C076E0972EAB
:105940006FE3F62EF822953619F450E4F52A07C0D5
:10595000963619F480E8F82A02C091109A94F7FE5E
:105960000BC09BE3991520F427E05CE3B52E0DC036
:10597000B92CB39427E009C0A7E0A91520F447E0AB
:10598000942E27E001C0292DBB24F6013496FD8713
:10599000EC87D6016D917D918D919C91AE014F5F09
:1059A0005F4F0B2D0E943F026C010981E02FF0E058
:1059B000FF87EE8700FF05C0FE85F3FD02C01DE2F4
:1059C00009C0F1FE02C01BE205C0F2FC02C010E0FB
:1059D00001C010E28E859F858C709070892B09F430
:1059E00044C0112311F483E001C084E0881510F055
:1059F00088240EC0881AF3FC0BC0D301ED91FC91F2
:105A00000190F081E02DC10160E209958A94A9F727
:105A1000112349F0D301ED91FC910190F081E02D2B
:105A2000C101612F0995BE85B3FF03C008E013E0F3
:105A300012C00CE013E00FC0E114F10409F0605251
:105A4000D301ED91FC910190F081E02DC101099508
:105A50000F5F1F4F05C0EF2CFF24B0E1EB22FF24A6
:105A6000F8016491662341F748C1F7FE13C0BC0CEE
:105A7000FE85F4FF04C08A81813309F4BA941B14B3
:105A80001CF0BB24B3942DC048E04B1550F538E012
:105A9000B32E27C0F6FC25C0892D90E08C159D05FE
:105AA0004CF05CEFC5165FEFD50624F080E8F82ACD
:105AB00001C09A94992049F0E2E0F0E0EC0FFD1F5C
:105AC000E90DF11D80818033A1F3F7FE0AC0B92CE6
:105AD000B394892D90E0C816D90614F0992401C01A
:105AE0009C18F7FC03C025E030E009C01C141D041D
:105AF0001CF021E030E003C096012F5F3F4F1123DF
:105B000011F02F5F3F4F992029F0892D90E00196E9
:105B1000280F391F882D90E02817390714F08824A2
:105B200001C0821A4F2C5524C20189709070892BB4
:105B300059F00CC0D301ED91FC910190F081E02D62
:105B4000C10160E209958A948820A1F7112349F0E8
:105B5000D301ED91FC910190F081E02DC101612F05
:105B6000099543FE0BC00CC0D301ED91FC9101904F
:105B7000F081E02DC10160E309958A948820A1F7A6
:105B8000F7FE51C08601D7FE02C000E010E07601AA
:105B90000894E11CF11CE01AF10AE1E0F0E0EC0FDE
:105BA000FD1FEE0EFF1E26014B185108892D90E0B7
:105BB000AA24BB24A81AB90AFFEF0F3F1F0749F414
:105BC000D301ED91FC910190F081E02DC1016EE2D5
:105BD0000995C016D10634F0401651061CF4F701A1
:105BE000608101C060E3015010400894E11CF11C89
:105BF0000A151B054CF0D301ED91FC910190F08149
:105C0000E02DC1010995D8CF0C151D0541F48A81FD
:105C1000863320F4853319F4BE85B4FF61E3D301E4
:105C2000ED91FC9165C06A81613309F00F7ED3016B
:105C3000ED91FC910190F081E02DC1010995992031
:105C4000E1F0D301ED91FC910190F081E02DC101D3
:105C50006EE2099512E0E1E0F0E0EC0FFD1FE10FCC
:105C6000F11D60811F5FD301ED91FC910190F081E6
:105C7000E02DC10109959A9471F7D301ED91FC9142
:105C80000190F081E02D44FC02C065E601C065E4AE
:105C9000C1010995D7FC05C0C114D10441F404FF2A
:105CA00006C0D094C194D108D3946DE201C06BE2D8
:105CB000D301ED91FC910190F081E02DC101099596
:105CC00060E305C06F5FE6EFFFEFCE0EDF1EFAE088
:105CD000CF16D104BCF7D301ED91FC910190F08176
:105CE000E02DC1010995D301ED91FC916C2D605D12
:105CF0000190F081E02DC1010995CC84DD8478C14B
:105D0000933631F0933799F0933509F061C023C091
:105D1000F601808189835E010894A11CB11C42E0D8
:105D200050E0C40ED51E21E0E22EF12C12C0D601A7
:105D3000AD90BC9016FD03C06FEF7FEF02C0692DE0
:105D400070E0E2E0F0E0CE0EDF1EC5010E94240408
:105D50007C011F7713C0D601AD90BC9016FD03C027
:105D60006FEF7FEF02C0692D70E0E2E0F0E0CE0E51
:105D7000DF1EC5010E9419047C01106813FF0BC0CF
:105D800023C0D301ED91FC910190F081E02DC10180
:105D900060E209958A94882D90E0E816F90688F368
:105DA00013C0F50117FD659117FF61915F01D301E4
:105DB000ED91FC910190F081E02DC10109958110D8
:105DC0008A940894E108F108E114F10451F710C134
:105DD000943611F0993699F517FF0AC0F601208123
:105DE00031814281538184E090E0C80ED91E0CC0FD
:105DF000D6018D919C919C01442737FD4095542FED
:105E0000E2E0F0E0CE0EDF1E9FE6F92EF12257FF12
:105E100009C050954095309521953F4F4F4F5F4FAA
:105E2000F0E8FF2ACA01B901AE014F5F5F4F2AE0D7
:105E300030E00E94E101E82E4B89E41A41C0953719
:105E400021F41F7E2AE030E01CC0197F9F3661F0EC
:105E5000903720F4983509F0CEC00FC0903739F054
:105E6000983709F0C8C004C028E030E00AC01061CB
:105E700014FD146020E130E004C014FD166020E140
:105E800032E017FF08C0D6016D917D918D919C91F4
:105E9000E4E0F0E008C0D6018D919C91BC0180E067
:105EA00090E0E2E0F0E0CE0EDF1EAE014F5F5F4F0C
:105EB0000E94E101E82EFB89EF1A8FE7F82EF1220C
:105EC000F6FE0BC04EEFF422E91438F4F4FE07C0DE
:105ED000F2FC05C05FEEF52202C01E2D01C0192D97
:105EE000F4FE0DC0FE01EE0DF11D8081803319F42A
:105EF00089EEF82208C01F5FF2FE05C003C08F2D97
:105F0000867809F01F5F0F2DF3FC18C0F0FE13C058
:105F1000181510F09E2C0FC09E2C980C911A182D5D
:105F20000AC0D301ED91FC910190F081E02DC101F7
:105F300060E209951F5F1815A0F304C0181510F44E
:105F4000811A01C0882404FF17C0D301ED91FC9190
:105F50000190F081E02DC10160E3099502FF29C0A5
:105F6000D301ED91FC910190F081E02D01FD02C083
:105F700068E712C068E510C0802F8678D1F001FF75
:105F800002C06BE201C060E2F7FC6DE2D301ED916B
:105F9000FC910190F081E02DC10109950AC0D30167
:105FA000ED91FC910190F081E02DC10160E3099534
:105FB0009A94E914A0F3EA94D301ED91FC91A1E045
:105FC000B0E0AC0FBD1FAE0DB11D0190F081E02D12
:105FD000C1016C910995EE2071F70AC0D301ED91D2
:105FE000FC910190F081E02DC10160E209958A9455
:105FF0008820A1F71DCC64960FB6F894DEBF0FBEC3
:10600000CDBFCF91DF911F910F91FF90EF90DF9067
:10601000CF90BF90AF909F908F907F906F905F9048
:106020004F903F902F900895F999FECF72BD61BDBA
:10603000F89A80B50895F999FECF1FBA72BD61BD77
:1060400040BD0FB6F894FA9AF99A0FBE08950F93CF
:10605000FC016115710511F480E011C021833283C8
:1060600043835483728761870170000F000F000F14
:106070008081877F802B82608B7F808381E00F917E
:106080000895CF93DF93EC010E94FC309B01AC019B
:106090008D819E81AF81B885281739074A075B0734
:1060A00028F4888184FD02C060E00DC089819A8156
:1060B000AB81BC81820F931FA41FB51F8D839E836C
:1060C000AF83B88761E0222757FD23953327442704
:1060D0005527922F91709295907F88818F7E892B82
:1060E0008883862FDF91CF910895CF93DF93EC01C2
:1060F000888182FF0FC0CE010E944130882351F079
:10610000E985FA85309709F00995888183FF02C0F7
:106110008B7F8883DF91CF910895CF93DF93EC013C
:1061200089859A85892BE1F089819A81AB81BC812F
:106130000097A105B105A1F00E94FC3029813A81A8
:106140004B815C81260F371F481F591F2D833E83CB
:106150004F835887888184608F7E888381E001C067
:1061600080E0DF91CF9108951F920F920FB60F92AA
:1061700011242F933F938F939F93AF93BF9380915D
:10618000A3069091A406A091A506B091A606309111
:10619000A7060196A11DB11D232F2D5F2D3720F0DD
:1061A0002D570196A11DB11D2093A7068093A3062C
:1061B0009093A406A093A506B093A60680919F068F
:1061C0009091A006A091A106B091A2060196A11DF2
:1061D000B11D80939F069093A006A093A106B09353
:1061E000A206BF91AF919F918F913F912F910F90F8
:1061F0000FBE0F901F9018958FB7F8942091A306AB
:106200003091A4064091A5065091A6068FBFB90112
:10621000CA0108959B01AC017FB7F89480919F0655
:106220009091A006A091A106B091A20666B5A89B88
:1062300005C06F3F19F00196A11DB11D7FBFBA2F98
:10624000A92F982F8827860F911DA11DB11D62E0EF
:10625000880F991FAA1FBB1F6A95D1F7BC012DC0DB
:10626000FFB7F89480919F069091A006A091A10697
:10627000B091A206E6B5A89B05C0EF3F19F00196C4
:10628000A11DB11DFFBFBA2FA92F982F88278E0FF0
:10629000911DA11DB11DE2E0880F991FAA1FBB1F10
:1062A000EA95D1F7861B970B885E9340C8F2215080
:1062B00030404040504068517C4F21153105410528
:1062C000510571F60895019739F0880F991F880FCD
:1062D000991F02970197F1F70895789484B5826029
:1062E00084BD84B5816084BD85B5826085BD85B57A
:1062F000816085BDEEE6F0E0808181608083E1E829
:10630000F0E0108280818260808380818160808360
:10631000E0E8F0E0808181608083E1EBF0E0808163
:1063200084608083E0EBF0E0808181608083EAE735
:10633000F0E08081846080838081826080838081BE
:10634000816080838081806880831092C10008957D
:106350001F920F920FB60F9211242F933F934F93DA
:106360005F936F937F938F939F93AF93BF93EF93BD
:10637000FF938091A8069091A906892B29F0E091BE
:10638000A806F091A9060995FF91EF91BF91AF91F1
:106390009F918F917F916F915F914F913F912F913D
:1063A0000F900FBE0F901F9018951F920F920FB66F
:1063B0000F9211242F933F934F935F936F937F938B
:1063C0008F939F93AF93BF93EF93FF938091AA0610
:1063D0009091AB06892B29F0E091AA06F091AB06CB
:1063E0000995FF91EF91BF91AF919F918F917F910F
:1063F0006F915F914F913F912F910F900FBE0F9032
:106400001F901895CF93DF93482F50E0CA018E5B01
:106410009C4FFC013491425D5C4FFA0184918823CA
:1064200069F190E0880F991FFC01E05FFC4FA59196
:10643000B491FC01E65EFC4FC591D491662351F402
:106440002FB7F8948C91932F909589238C93888102
:1064500089230BC0623061F42FB7F8948C91932F8D
:10646000909589238C938881832B88832FBF06C0C6
:106470009FB7F8948C91832B8C939FBFDF91CF9122
:106480000895482F50E0CA018A5A9C4FFC0124917C
:10649000CA018E5B9C4FFC019491425D5C4FFA01F6
:1064A0003491332309F440C0222351F1233071F099
:1064B000243028F42130A1F0223011F514C0263008
:1064C000B1F02730C1F02430D9F404C080918000AD
:1064D0008F7703C0809180008F7D8093800010C0F3
:1064E00084B58F7702C084B58F7D84BD09C080914B
:1064F000B0008F7703C08091B0008F7D8093B00093
:10650000E32FF0E0EE0FFF1FE65EFC4FA591B49184
:106510002FB7F894662321F48C919095892302C0BB
:106520008C91892B8C932FBF0895CF92DF92EF929D
:10653000FF920F931F93CF93DF937C016B018A012E
:10654000C0E0D0E00FC0D6016D916D01D701ED9193
:10655000FC910190F081E02DC7010995C80FD91F6A
:10656000015010400115110571F7CE01DF91CF9157
:106570001F910F91FF90EF90DF90CF900895CF93F0
:10658000DF930E946D310E946327C0E0D0E00E943B
:1065900043292097E1F30E940000F9CF5058BB2710
:1065A000AA270ED041C201D230F006D220F031F439
:1065B0009F3F11F41EF4C0C10EF4E095E7FBB6C195
:1065C000E92F54D280F3BA1762077307840795073F
:1065D00018F071F49EF56CC20EF4E0950B2EBA2FF4
:1065E000A02D0B01B90190010C01CA01A0011124D9
:1065F000FF27591B99F0593F50F4503E68F11A1685
:10660000F040A22F232F342F4427585FF3CF469515
:1066100037952795A795F0405395C9F77EF41F1637
:10662000BA0B620B730B840BBAF09150A1F0FF0F01
:10663000BB1F661F771F881FC2F70EC0BA0F621FED
:10664000731F841F48F4879577956795B795F795DD
:106650009E3F08F0B3CF9395880F08F09927EE0F6F
:10666000979587950895A1D158F080E891E009F4B5
:106670009EEFA2D128F040E851E059F45EEF09C046
:106680005BC116C2E92FE078F1D168F3092E052A23
:10669000C1F3261737074807590738F00E2E07F8B9
:1066A000E02569F0E025E0640AC0EF6307F8009494
:1066B00007FADB01B9019D01DC01CA01AD01EF93CD
:1066C0004AD0B2D10AD05F91552331F02BED3FE093
:1066D00049E450FD49EC63CF0895DF93DD27B92FDE
:1066E000BF7740E85FE31616170648075B0710F40C
:1066F000D92FE9D19F938F937F936F93BCD2E8E614
:10670000F0E01DD191D12F913F914F915F91EED14A
:10671000DD2349F09058A2EA2AED3FE049EC5FE31F
:10672000D0785D274DDFDF917FC1DCD008F481E0B8
:1067300008954AD1E39589C10CD076C13DD140F08E
:1067400034D130F021F45F3F19F0F0C05111B1C1E4
:10675000F3C08CD198F39923C9F35523B1F3951B5A
:10676000550BBB27AA2762177307840738F09F5F72
:106770005F4F220F331F441FAA1FA9F333D00E2EE1
:106780003AF0E0E830D091505040E695001CCAF74E
:1067900029D0FE2F27D0660F771F881FBB1F261713
:1067A00037074807AB07B0E809F0BB0B802DBF01E6
:1067B000FF2793585F4F2AF09E3F510568F0B6C0FF
:1067C00078C15F3FECF3983EDCF38695779567954B
:1067D000B795F7959F5FC9F7880F911D9695879597
:1067E00097F90895E1E0660F771F881FBB1F6217B6
:1067F00073078407BA0720F0621B730B840BBA0B74
:10680000EE1F88F7E095089504D06894B11151C146
:10681000089534D188F09F5790F0B92F9927B75138
:10682000A0F0D1F0660F771F881F991F1AF0BA9554
:10683000C9F712C0B13081F03BD1B1E0089538C141
:10684000672F782F8827B85F39F0B93FCCF386954A
:1068500077956795B395D9F73EF4909580957095A7
:1068600061957F4F8F4F9F4F0895E89409C097FB24
:106870003EF490958095709561957F4F8F4F9F4F17
:106880009923A9F0F92F96E9BB279395F69587955B
:1068900077956795B795F111F8CFFAF4BB0F11F41E
:1068A00060FF1BC06F5F7F4F8F4F9F4F16C08823C5
:1068B00011F096E911C0772321F09EE8872F762FFB
:1068C00005C0662371F096E8862F70E060E02AF03C
:1068D0009A95660F771F881FDAF7880F9695879528
:1068E00097F90895990F0008550FAA0BE0E8FEEFFD
:1068F00016161706E807F907C0F012161306E40784
:10690000F50798F0621B730B840B950B39F40A267C
:1069100061F0232B242B252B21F408950A2609F45A
:10692000A140A6958FEF811D811D089597F99F675E
:1069300080E870E060E008959FEF80EC0895DF93B9
:10694000CF931F930F93FF92EF92DF927B018C0105
:10695000689405C0DA2EEF01C9D0FE01E894A59134
:106960002591359145915591AEF3EF0129DEFE0158
:106970009701A801DA9479F7DF90EF90FF900F91DB
:106980001F91CF91DF9108959F938F937F936F9382
:10699000FF93EF939B01AC019DD0EF91FF91CFDF6F
:1069A0002F913F914F915F9195C000240A94161644
:1069B000170618060906089500240A9412161306ED
:1069C000140605060895B8CF59D0E8F3E894EFEF20
:1069D000BB273FE048EC5FE76B3D730784079507F3
:1069E00008F1FF279F57B25A6A4D7F40894CF0400B
:1069F00032F4BE556542704F8643FF4F0894EE1F38
:106A0000915030F0BB0F661F771F881FFF1FEBCF21
:106A10009EE7882332F0BB0F661F771F881F9A9569
:106A2000C1F79395E09565C1092E0394000C11F40C
:106A3000882352F0BB0F40F4BF2B11F460FF04C059
:106A40006F5F7F4F8F4F9F4F0895EF93E0FF06C01A
:106A5000A2EA2AED3FE049EC5FEBB2DDE5DF0F9003
:106A6000039401FC9058E5E9F0E08ECF57FD905873
:106A7000440F551F59F05F3F71F04795880F97FB02
:106A8000991F61F09F3F79F08795089512161306BC
:106A90001406551FF2CF4695F1DF08C016161706EB
:106AA0001806991FF1CF8695710561050894089520
:106AB000E894BB2766277727CB0197F9089512DF63
:106AC00008F48FEF08959B01AC0160E070E080E86E
:106AD0009FE332CE0BD0A8CF68DF28F06DDF18F02F
:106AE000952309F023CF28CF1124E3CFBFDFA0F3F4
:106AF000959FD1F3950F50E0551F629FF001729F53
:106B0000BB27F00DB11D639FAA27F00DB11DAA1F71
:106B1000649F6627B00DA11D661F829F2227B00DBE
:106B2000A11D621F739FB00DA11D621F839FA00D49
:106B3000611D221F749F3327A00D611D231F849F99
:106B4000600D211D822F762F6A2F11249F575040F0
:106B50008AF0E1F088234AF0EE0FFF1FBB1F661F8B
:106B6000771F881F91505040A9F79E3F510570F044
:106B7000DDCE9FCF5F3FECF3983EDCF386957795B3
:106B80006795B795F795E7959F5FC1F7FE2B880F3F
:106B9000911D9695879597F9089570DFE0F09E37DF
:106BA000D8F09639B8F49E3848F4672F782F8827A4
:106BB000985FF9CF86957795679593959539D0F33A
:106BC000B62FB1706B0F711D811D20F487957795DD
:106BD0006795939573C08DC06CCF11F40EF4ACCE55
:106BE00088C04CDFD0F39923D9F3CEF39F57550BD0
:106BF00087FF8FD056959795B0E020F4660F771FEA
:106C0000881FBB1F1F930F9300249001A0018001D8
:106C1000F001A0E80E0F1F1F0A1E511D601B710B13
:106C20008009B50B48F4600F711F801DB51F0E1B46
:106C30001F0B0A0A510907C02E0F3F1F4A1F0E0FD4
:106C40001F1F0A1E511D660F771F881FBB1FA695A9
:106C5000F795E795F8F60617170708065B07211D55
:106C6000311D411D0F911F91B901842F9158880F3B
:106C70009695879508959B01AC012CCFDF93D92F72
:106C8000A3DEE695D7952AED3FE049E45FE3B33A0A
:106C90006207730784079507D7952AF0A2EA49ECA3
:106CA00090688EDCC1DEE3EBF0E06EDEDD0F0BF012
:106CB0000ADFDD0F0BF49058DF910895882371F4FB
:106CC000772321F09850872B762F07C0662311F485
:106CD00099270DC09051862B70E060E02AF09A95BC
:106CE000660F771F881FDAF7880F9695879597F9B3
:106CF00008959F3F49F0915028F4869577956795C0
:106D0000B7959F5F80389F4F880F9695879597F925
:106D1000089591505040660F771F881FD2F708954D
:106D2000AA1BBB1B51E107C0AA1FBB1FA617B707B1
:106D300010F0A61BB70B881F991F5A95A9F78095CD
:106D40009095BC01CD01089597FB092E07260AD026
:106D500077FD04D0E5DF06D000201AF47095619528
:106D60007F4F0895F6F7909581959F4F0895A1E282
:106D70001A2EAA1BBB1BFD010DC0AA1FBB1FEE1FB5
:106D8000FF1FA217B307E407F50720F0A21BB30B00
:106D9000E40BF50B661F771F881F991F1A9469F77C
:106DA00060957095809590959B01AC01BD01CF01D8
:106DB000089597FB092E05260ED057FD04D0D7DF86
:106DC0000AD0001C38F450954095309521953F4FDE
:106DD0004F4F5F4F0895F6F79095809570956195A8
:106DE0007F4F8F4F9F4F0895EE0FFF1F0590F49137
:086DF000E02D0994F894FFCF97
:106DF80025630025632563002563253269256325FE
:106E08003032697C25632532692563253032690073
:106E180025352E3066256300256325312E356625F8
:106E280063002563253569256300256325352E32E2
:106E3800662563006D616E007374310073743200EF
:106E480073743300737434007374350073743600CC
:106E580070682000636C200076722000686C200047
:106E680061702000727462006C616E0070702000A6
:106E7800706F69006163200000617420002563253C
:106E88007300256325332E30692563002534692571
:106E980063256300256325336925630025737C25F5
:106EA80063257325630020C0C0C0C0C0C7C0C0C070
:106EB800C0C0200025342E306625630025632533A5
:106EC8002E3066256300256325352E306625630040
:106ED80025632531312E36667C25632531312E36E2
:106EE800660025632532690025332E316625630047
:106EF8002020202020202020202020200020206466
:106F0800697361726D6564202000206E6F2074655E
:106F18006C20636F6D2000206E6F20677073206691
:106F280069782000202062617474206C6F772020BB
:106F38000062617474207761726E696E67006261C5
:106F48007474637269746963616C0020626174743B
:106F5800206572726F7220006C696E6B20717561AA
:106F68006C697479006D6167207761726E696E670C
:106F7800006D616720637269746963616C00206DDC
:106F8800616720206572726F7220002573002000EF
:106F9800B0060000E803E803E803E8039DFF016486
:106FA8000000000077059532750478047B047E04A0
:106FB8004F2900070E091C1B1215383F36312423B0
:106FC8002A2D70777E796C6B6265484F4641545321
:106FD8005A5DE0E7EEE9FCFBF2F5D8DFD6D1C4C391
:106FE800CACD90979E998C8B8285A8AFA6A1B4B381
:106FF800BABDC7C0C9CEDBDCD5D2FFF8F1F6E3E4F1
:10700800EDEAB7B0B9BEABACA5A28F8881869394E0
:107018009D9A2720292E3B3C35321F181116030450
:107028000D0A5750595E4B4C45426F686166737440
:107038007D7A898E878095929B9CB1B6BFB8ADAAA0
:10704800A3A4F9FEF7F0E5E2EBECC1C6CFC8DDDAA0
:10705800D3D4696E676075727B7C51565F584D4A10
:107068004344191E171005020B0C21262F283D3A00
:1070780033344E49404752555C5B7671787F6A6D70
:1070880064633E39303722252C2B0601080F1A1D60
:107098001413AEA9A0A7B2B5BCBB9691989F8A8DD0
:1070A8008483DED9D0D7C2C5CCCBE6E1E8EFFAFDC0
:1070B800F4F3C2C0C0C1C0C0C1C0C0C4C0C0C1C058
:1070C800C0C1C0C0C3C0C0C1C0C0C1C0C0C5C0C0AD
:1070D800C1C0C0C1C0C000000000652A9532D629D1
:0E70E800062A362A532AEC297429BA2A2A2BA2
:00000001FF
